:020000040000FA
:06000000B4EF37F012001E
:020006001200E6
:0600080022EF00F01200DF
:02000E00A6B298
:04001000FED7120005
:020014001200D8
:020016000100E7
:06001800DAEF00F0120017
:02001E000300DD
:10002000DE6F0000980100001D000000B16F0000AD
:100030006B0100002D00000016000000F40000001D
:0400400002000000BA
:0C004400DACFE4FFE2CFDAFFE9CFE4FFFF
:10005000EACFE4FFF6CFE4FFF7CFE4FFF8CFE4FF09
:10006000F5CFE4FFF3CFE4FFF4CFE4FFFACFE4FFF2
:10007000FBCFE4FF00EE00F0140EE80403E3EECF44
:10008000E4FFFBD700EE14F00C0EE80403E3EECF20
:10009000E4FFFBD7E65201EC1BF0A1A263D0A192D2
:1000A000F70EB36EB26A010EE06E9D29070B9D6FCD
:1000B0000AE1080E9C253F0B9C6F05E19E2B070B68
:1000C0009E6F01E19B6B9C51030D000EF324E96EC2
:1000D000020EF420EA6E986B996B9A6B9D29EE6084
:1000E0009881EE609981EE609A81EE609883EE606F
:1000F0009983EE609A83EE609885EE609985EE6054
:100100009A85EE609887EE609987EE609A87EE6038
:100110009889EE609989EE609A89EE60988BEE601E
:10012000998BEE609A8BEE60988DEE60998DEE6003
:100130009A8DEE60988FEE60998FEE609A8F010134
:100140009C51E840E840E8401F0BE66E9AC1E6FF8C
:1001500099C1E6FF98C1E6FF82EC18F0E552E5523E
:10016000E552E552E55200EE1FF00C0EE80403E301
:10017000E5CFEDFFFBD700EE13F0140EE80403E328
:10018000E5CFEDFFFBD7E5CFFBFFE5CFFAFFE5CFEE
:10019000F4FFE5CFF3FFE5CFF5FFE5CFF8FFE5CFBF
:1001A000F7FFE5CFF6FFE5CFEAFFE5CFE9FFE5CFC3
:1001B000DAFF1100D8CFE4FFE0CFE4FFE46EDACF3E
:1001C000E4FFE65201019B6BE552E5CFDAFFE55013
:1001D000E5CFE0FFE5CFD8FF1000D9CFE6FFE1CFB4
:1001E000D9FFE652DF6AFCEC17F02FEC1DF04FEC64
:1001F00032F0960EE66E6C0EE66E000EE66E000EA7
:10020000E66E010EE66EE8EC34F0146E050EE15E6B
:100210001450000EE66E010EE66E57EC32F0E55219
:10022000E5527E0EE66E6C0EE66E000EE66E000E79
:10023000E66E010EE66EE8EC34F0146E050EE15E3B
:100240001450000EE66E010EE66E57EC32F0E552E9
:10025000E552000EE66EE66A1EEC37F0E552E55216
:100260000101A76F6D0E146E580E156E000E166EFE
:10027000ACC117F0186A196A17AE02D0186819686D
:1002800014501724F36E15501820F46E16501920D0
:10029000F86EF4CFF7FFF3CFF6FF0800F5CF50F17B
:1002A000E0EC18F001019B51FBE1A605F9E1010E1C
:1002B0009B6FDF2A8050100B05E08050200B02E07E
:1002C000B05103E0C3EC15F0EBD7AB51D880DF544D
:1002D000E7E2DF6A32D8E4D7D9CFE6FFE1CFD9FF32
:1002E000FE0EDB500DE0080E166EFD0EDB28165CD0
:1002F00002E2080E02D0FD0EDB28156AF36E17D05D
:10030000166AFD0EDB04E76E1618E8AE02D016344E
:1003100003D0E750D880165402E2000E02D0FD0E42
:10032000DB04146E156A14BE156814C0F3FF15C003
:10033000F4FFE552E7CFD9FF1200D9CFE6FFE1CFB6
:10034000D9FF050EE1260101AD51AE1154E1ADC159
:1003500014F0AEC115F0AD2B000EAE23166AACC181
:10036000E9FFEA6AE9BEEA68030EEA02F3CFEAFFB0
:10037000E902F3CFE9FFF450EA266B0EE926010EFD
:10038000EA22EE501424F36EEE501520F46EEE5077
:100390001620F86EF4CFF7FFF3CFF6FF0800F5CF85
:1003A000A9F1ADC114F0AEC115F0AD2B000EAE2316
:1003B000166AACC1E9FFEA6AE9BEEA68030EEA021E
:1003C000F3CFEAFFE902F3CFE9FFF450EA266B0E20
:1003D000E926010EEA22EE501424F36EEE501520A9
:1003E000F46EEE501620F86EF4CFF7FFF3CFF6FF61
:1003F0000800F5CFABF1A951040A02E1E9EF0DF0D5
:10040000060A02E114EF06F0010A02E114EF06F019
:10041000020A02E079EF15F0DF6A080EDF5C02E302
:1004200079EF15F0ADC114F0AEC115F0166AACC18C
:10043000E9FFEA6AE9BEEA68030EEA02F3CFEAFFDF
:10044000E902F3CFE9FFF450EA266B0EE926010E2C
:10045000EA22EE501424F36EEE501520F46EEE50A6
:100460001620F86EF4CFF7FFF3CFF6FF0800020E68
:10047000F5CFDBFF080EDF02F350E66ED950030F15
:10048000E96EDACFEAFFE552E750EE6EED6A020E52
:10049000DB50800B02E0070E01D0000EE66E030E6B
:1004A000DBCFE9FF040EDBCFEAFF030EEA02F3CF56
:1004B000EAFFE902F3CFE9FFF450EA26000EE9264D
:1004C000020EEA22E552E750EF6E020EDB50400BBF
:1004D00002E0070E01D0000EE66E010EE76E030E7D
:1004E000DBCFE9FF040EDBCFEAFFE750E926000E81
:1004F000EA22030EEA02F3CFEAFFE902F3CFE9FFB3
:10050000F450EA26000EE926020EEA22E552E750F0
:10051000EF6E020EDB50200B02E0070E01D0000E42
:10052000E66E020EE76E030EDBCFE9FF040EDBCFB3
:10053000EAFFE750E926000EEA22030EEA02F3CFB3
:10054000EAFFE902F3CFE9FFF450EA26000EE926BC
:10055000020EEA22E552E750EF6E020EDB50100B5E
:1005600002E0070E01D0000EE66E030EE76EDBCF51
:10057000E9FF040EDBCFEAFFE750E926000EEA228E
:10058000030EEA02F3CFEAFFE902F3CFE9FFF450EA
:10059000EA26000EE926020EEA22E552E750EF6E47
:1005A000020EDB50080B02E0070E01D0000EE66ED3
:1005B000040EE76E030EDBCFE9FF040EDBCFEAFF8C
:1005C000E750E926000EEA22030EEA02F3CFEAFF23
:1005D000E902F3CFE9FFF450EA26000EE926020E05
:1005E000EA22E552E750EF6E020EDB50040B02E008
:1005F000070E01D0000EE66E050EE76E030EDBCF90
:10060000E9FF040EDBCFEAFFE750E926000EEA22FD
:10061000030EEA02F3CFEAFFE902F3CFE9FFF45059
:10062000EA26000EE926020EEA22E552E750EF6EB6
:10063000020EDB50020B02E0070E01D0000EE66E48
:10064000060EE76E030EDBCFE9FF040EDBCFEAFFF9
:10065000E750E926000EEA22030EEA02F3CFEAFF92
:10066000E902F3CFE9FFF450EA26000EE926020E74
:10067000EA22E552E750EF6E020EDB50010B02E07A
:10068000070E01D0000EE66E070EE76E030EDBCFFD
:10069000E9FF040EDBCFEAFFE750E926000EEA226D
:1006A000030EEA02F3CFEAFFE902F3CFE9FFF450C9
:1006B000EA26000EE926020EEA22E552E750EF6E26
:1006C000AD2B000EAE23ADC114F0AEC115F0166A0D
:1006D000ACC1E9FFEA6AE9BEEA68030EEA02F3CFB9
:1006E000EAFFE902F3CFE9FFF450EA266B0EE926B0
:1006F000010EEA22EE501424F36EEE501520F46E33
:10070000EE501620F86EF4CFF7FFF3CFF6FF080097
:10071000020EF5CFDBFFDB50800B02E0070E01D0AD
:10072000000EE66E030EDBCFE9FF040EDBCFEAFF1F
:10073000030EEA02F3CFEAFFE902F3CFE9FFF45038
:10074000EA26000EE926020EEA22EE52E552E750B2
:10075000EF6E020EDB50400B02E0070E01D0000EE0
:10076000E66E010EE76E030EDBCFE9FF040EDBCF72
:10077000EAFFE750E926000EEA22030EEA02F3CF71
:10078000EAFFE902F3CFE9FFF450EA26000EE9267A
:10079000020EEA22EE52E552E750EF6E020EDB50F7
:1007A000200B02E0070E01D0000EE66E020EE76E8F
:1007B000030EDBCFE9FF040EDBCFEAFFE750E926AB
:1007C000000EEA22030EEA02F3CFEAFFE902F3CFBA
:1007D000E9FFF450EA26000EE926020EEA22EE5264
:1007E000E552E750EF6E020EDB50100B02E0070EF1
:1007F00001D0000EE66E030EE76EDBCFE9FF040EBC
:10080000DBCFEAFFE750E926000EEA22030EEA02F8
:10081000F3CFEAFFE902F3CFE9FFF450EA26000E36
:10082000E926020EEA22EE52E552E750EF6E020E82
:10083000DB50080B02E0070E01D0000EE66E040E3E
:10084000E76E030EDBCFE9FF040EDBCFEAFFE750D4
:10085000E926000EEA22030EEA02F3CFEAFFE902DC
:10086000F3CFE9FFF450EA26000EE926020EEA2251
:10087000EE52E552E750EF6E020EDB50040B02E041
:10088000070E01D0000EE66E050EE76E030EDBCFFD
:10089000E9FF040EDBCFEAFFE750E926000EEA226B
:1008A000030EEA02F3CFEAFFE902F3CFE9FFF450C7
:1008B000EA26000EE926020EEA22EE52E552E75041
:1008C000EF6E020EDB50020B02E0070E01D0000EAD
:1008D000E66E060EE76E030EDBCFE9FF040EDBCFFC
:1008E000EAFFE750E926000EEA22030EEA02F3CF00
:1008F000EAFFE902F3CFE9FFF450EA26000EE92609
:10090000020EEA22EE52E552E750EF6E020EDB5085
:10091000010B02E0070E01D0000EE66E070EE76E37
:10092000030EDBCFE9FF040EDBCFEAFFE750E92639
:10093000000EEA22030EEA02F3CFEAFFE902F3CF48
:10094000E9FFF450EA26000EE926020EEA22EE52F2
:10095000E552E750EF6EAD2B000EAE23ADC114F0A3
:10096000AEC115F0166AACC1E9FFEA6AE9BEEA68F1
:10097000030EEA02F3CFEAFFE902F3CFE9FFF450F6
:10098000EA266B0EE926010EEA22EE501424F36EDD
:10099000EE501520F46EEE501620F86EF4CFF7FFEF
:1009A000F3CFF6FF0800020EF5CFDBFFDB50800B24
:1009B00002E0070E01D0000EE66E030EDBCFE9FF6A
:1009C000040EDBCFEAFF030EEA02F3CFEAFFE902EF
:1009D000F3CFE9FFF450EA26000EE926020EEA22E0
:1009E000020EE926000EEA22E552E750EF6E020EF3
:1009F000DB50400B02E0070E01D0000EE66E010E48
:100A0000E76E030EDBCFE9FF040EDBCFEAFFE75012
:100A1000E926000EEA22030EEA02F3CFEAFFE9021A
:100A2000F3CFE9FFF450EA26000EE926020EEA228F
:100A3000020EE926000EEA22E552E750EF6E020EA2
:100A4000DB50200B02E0070E01D0000EE66E020E16
:100A5000E76E030EDBCFE9FF040EDBCFEAFFE750C2
:100A6000E926000EEA22030EEA02F3CFEAFFE902CA
:100A7000F3CFE9FFF450EA26000EE926020EEA223F
:100A8000020EE926000EEA22E552E750EF6E020E52
:100A9000DB50100B02E0070E01D0000EE66E030ED5
:100AA000E76EDBCFE9FF040EDBCFEAFFE750E92674
:100AB000000EEA22030EEA02F3CFEAFFE902F3CFC7
:100AC000E9FFF450EA26000EE926020EEA22020EA1
:100AD000E926000EEA22E552E750EF6E020EDB50E7
:100AE000080B02E0070E01D0000EE66E040EE76E62
:100AF000030EDBCFE9FF040EDBCFEAFFE750E92668
:100B0000000EEA22030EEA02F3CFEAFFE902F3CF76
:100B1000E9FFF450EA26000EE926020EEA22020E50
:100B2000E926000EEA22E552E750EF6E020EDB5096
:100B3000040B02E0070E01D0000EE66E050EE76E14
:100B4000030EDBCFE9FF040EDBCFEAFFE750E92617
:100B5000000EEA22030EEA02F3CFEAFFE902F3CF26
:100B6000E9FFF450EA26000EE926020EEA22020E00
:100B7000E926000EEA22E552E750EF6E020EDB5046
:100B8000020B02E0070E01D0000EE66E060EE76EC5
:100B9000030EDBCFE9FF040EDBCFEAFFE750E926C7
:100BA000000EEA22030EEA02F3CFEAFFE902F3CFD6
:100BB000E9FFF450EA26000EE926020EEA22020EB0
:100BC000E926000EEA22E552E750EF6E020EDB50F6
:100BD000010B02E0070E01D0000EE66E070EE76E75
:100BE000030EDBCFE9FF040EDBCFEAFFE750E92677
:100BF000000EEA22030EEA02F3CFEAFFE902F3CF86
:100C0000E9FFF450EA26000EE926020EEA22020E5F
:100C1000E926000EEA22E552E750EF6EAD2B000EFA
:100C2000AE23DF2A0DEF02F0B15101E0FCD0030E3C
:100C3000A95D08E14A0EE66E490EE66E40EC37F01B
:100C4000E552E552DF6A080EDF5C01E3C1D0020E17
:100C50000101A95D01E090D0ADC114F0AEC115F065
:100C6000AD2B000EAE23166AACC1E9FFEA6AE9BEFD
:100C7000EA68030EEA02F3CFEAFFE902F3CFE9FFE5
:100C8000F450EA266B0EE926010EEA22EE501424F7
:100C9000F36EEE501520F46EEE501620F86EF4CF81
:100CA000F7FFF3CFF6FF0800F550E66EDF50EA6A73
:100CB000510FE96E010EEA22E552E750EF6EADC129
:100CC00014F0AEC115F0AD2B000EAE23166AACC108
:100CD000E9FFEA6AE9BEEA68030EEA02F3CFEAFF37
:100CE000E902F3CFE9FFF450EA266B0EE926010E84
:100CF000EA22EE501424F36EEE501520F46EEE50FE
:100D00001620F86EF4CFF7FFF3CFF6FF0800F5508A
:100D1000E66EDF50EA6A590FE96E010EEA22E552EB
:100D2000E750EF6EADC114F0AEC115F0AD2B000E63
:100D3000AE23166AACC1E9FFEA6AE9BEEA68030EAF
:100D4000EA02F3CFEAFFE902F3CFE9FFF450EA2623
:100D50006B0EE926010EEA22EE501424F36EEE50DB
:100D60001520F46EEE501620F86EF4CFF7FFF3CF97
:100D7000F6FF0800F55020D0030EA95D27E19AEC9C
:100D800017F0F350E66EDF50EA6A510FE96E010E7C
:100D9000EA22E552E750EF6E9AEC17F0F350E66E58
:100DA000DF50EA6A590FE96E010EEA22E552E75078
:100DB000EF6E9AEC17F0F350E66EDF50EA6A610FBF
:100DC000E96E010EEA22E552E750EF6EDF2A3BD7CB
:100DD0000101ADC114F0AEC115F0AD2B000EAE2374
:100DE000166AACC1E9FFEA6AE9BEEA68030EEA02E4
:100DF000F3CFEAFFE902F3CFE9FFF450EA266B0EE6
:100E0000E926010EEA22EE501424F36EEE5015206E
:100E1000F46EEE501620F86EF4CFF7FFF3CFF6FF26
:100E20000800F5CFAAF1DF6A080EDF5C02E3DFEF0E
:100E30000DF0080EDF02F350E66ED950030FE96E95
:100E4000DACFEAFFE552E750EE6EED6A030EDBCF34
:100E5000E9FF040EDBCFEAFF030EEA02F3CFEAFF5D
:100E6000E902F3CFE9FFF450EA26000EE926020E6C
:100E7000EA22EF50E66EDF50EA6A510FE96E010E8A
:100E8000EA22EF50800BE66E6CEC01F0E552E55281
:100E9000F350E66E030EDBCFE9FF040EDBCFEAFF73
:100EA000030EEA02F3CFEAFFE902F3CFE9FFF450C1
:100EB000EA26000EE926020EEA22E552E750EF6E1E
:100EC000010EE76E030EDBCFE9FF040EDBCFEAFF76
:100ED000E750E926000EEA22030EEA02F3CFEAFF0A
:100EE000E902F3CFE9FFF450EA26000EE926020EEC
:100EF000EA22EF50E66EDF50EA6A510FE96E010E0A
:100F0000EA22EF50400BE66E6CEC01F0E552E55240
:100F1000F350E66E010EE76E030EDBCFE9FF040E21
:100F2000DBCFEAFFE750E926000EEA22030EEA02D1
:100F3000F3CFEAFFE902F3CFE9FFF450EA26000E0F
:100F4000E926020EEA22E552E750EF6E020EE76E46
:100F5000030EDBCFE9FF040EDBCFEAFFE750E92603
:100F6000000EEA22030EEA02F3CFEAFFE902F3CF12
:100F7000E9FFF450EA26000EE926020EEA22EF50BD
:100F8000E66EDF50EA6A510FE96E010EEA22EF5079
:100F9000200BE66E6CEC01F0E552E552F350E66E84
:100FA000020EE76E030EDBCFE9FF040EDBCFEAFF94
:100FB000E750E926000EEA22030EEA02F3CFEAFF29
:100FC000E902F3CFE9FFF450EA26000EE926020E0B
:100FD000EA22E552E750EF6E030EE76EDBCFE9FF42
:100FE000040EDBCFEAFFE750E926000EEA22030EEB
:100FF000EA02F3CFEAFFE902F3CFE9FFF450EA2671
:10100000000EE926020EEA22EF50E66EDF50EA6A91
:10101000510FE96E010EEA22EF50100BE66E6CECF8
:1010200001F0E552E552F350E66E030EE76EDBCFBA
:10103000E9FF040EDBCFEAFFE750E926000EEA22C3
:10104000030EEA02F3CFEAFFE902F3CFE9FFF4501F
:10105000EA26000EE926020EEA22E552E750EF6E7C
:10106000040EE76E030EDBCFE9FF040EDBCFEAFFD1
:10107000E750E926000EEA22030EEA02F3CFEAFF68
:10108000E902F3CFE9FFF450EA26000EE926020E4A
:10109000EA22EF50E66EDF50EA6A510FE96E010E68
:1010A000EA22EF50080BE66E6CEC01F0E552E552D7
:1010B000F350E66E040EE76E030EDBCFE9FF040E7D
:1010C000DBCFEAFFE750E926000EEA22030EEA0230
:1010D000F3CFEAFFE902F3CFE9FFF450EA26000E6E
:1010E000E926020EEA22E552E750EF6E050EE76EA2
:1010F000030EDBCFE9FF040EDBCFEAFFE750E92662
:10110000000EEA22030EEA02F3CFEAFFE902F3CF70
:10111000E9FFF450EA26000EE926020EEA22EF501B
:10112000E66EDF50EA6A510FE96E010EEA22EF50D7
:10113000040BE66E6CEC01F0E552E552F350E66EFE
:10114000050EE76E030EDBCFE9FF040EDBCFEAFFEF
:10115000E750E926000EEA22030EEA02F3CFEAFF87
:10116000E902F3CFE9FFF450EA26000EE926020E69
:10117000EA22E552E750EF6E060EE76E030EDBCF74
:10118000E9FF040EDBCFEAFFE750E926000EEA2272
:10119000030EEA02F3CFEAFFE902F3CFE9FFF450CE
:1011A000EA26000EE926020EEA22EF50E66EDF5034
:1011B000EA6A510FE96E010EEA22EF50020BE66E69
:1011C0006CEC01F0E552E552F350E66E060EE76E68
:1011D000030EDBCFE9FF040EDBCFEAFFE750E92681
:1011E000000EEA22030EEA02F3CFEAFFE902F3CF90
:1011F000E9FFF450EA26000EE926020EEA22E55243
:10120000E750EF6E070EE76E030EDBCFE9FF040E2B
:10121000DBCFEAFFE750E926000EEA22030EEA02DE
:10122000F3CFEAFFE902F3CFE9FFF450EA26000E1C
:10123000E926020EEA22EF50E66EDF50EA6A510F0D
:10124000E96E010EEA22EF50010BE66E6CEC01F044
:10125000E552E552F350E66E070EE76E030EDBCF64
:10126000E9FF040EDBCFEAFFE750E926000EEA2291
:10127000030EEA02F3CFEAFFE902F3CFE9FFF450ED
:10128000EA26000EE926020EEA22E552E750EF6E4A
:10129000030EDBCFE9FF040EDBCFEAFF030EEA0209
:1012A000F3CFEAFFE902F3CFE9FFF450EA26000E9C
:1012B000E926020EEA22EE52EF50E66EDF50EA6AAD
:1012C000590FE96E010EEA22EF50800BE66E6CECCE
:1012D00001F0E552E552F350E66E030EDBCFE9FF75
:1012E000040EDBCFEAFF030EEA02F3CFEAFFE902C6
:1012F000F3CFE9FFF450EA26000EE926020EEA22B7
:10130000EE52E552E750EF6E010EE76E030EDBCFB3
:10131000E9FF040EDBCFEAFFE750E926000EEA22E0
:10132000030EEA02F3CFEAFFE902F3CFE9FFF4503C
:10133000EA26000EE926020EEA22EE52EF50E66E91
:10134000DF50EA6A590FE96E010EEA22EF50400BB6
:10135000E66E6CEC01F0E552E552F350E66E010EDC
:10136000E76E030EDBCFE9FF040EDBCFEAFFE750A9
:10137000E926000EEA22030EEA02F3CFEAFFE902B1
:10138000F3CFE9FFF450EA26000EE926020EEA2226
:10139000EE52E552E750EF6E020EE76E030EDBCF22
:1013A000E9FF040EDBCFEAFFE750E926000EEA2250
:1013B000030EEA02F3CFEAFFE902F3CFE9FFF450AC
:1013C000EA26000EE926020EEA22EE52EF50E66E01
:1013D000DF50EA6A590FE96E010EEA22EF50200B46
:1013E000E66E6CEC01F0E552E552F350E66E020E4B
:1013F000E76E030EDBCFE9FF040EDBCFEAFFE75019
:10140000E926000EEA22030EEA02F3CFEAFFE90220
:10141000F3CFE9FFF450EA26000EE926020EEA2295
:10142000EE52E552E750EF6E030EE76EDBCFE9FFB9
:10143000040EDBCFEAFFE750E926000EEA22030E96
:10144000EA02F3CFEAFFE902F3CFE9FFF450EA261C
:10145000000EE926020EEA22EE52EF50E66EDF5051
:10146000EA6A590FE96E010EEA22EF50100BE66EA0
:101470006CEC01F0E552E552F350E66E030EE76EB8
:10148000DBCFE9FF040EDBCFEAFFE750E926000ED1
:10149000EA22030EEA02F3CFEAFFE902F3CFE9FF03
:1014A000F450EA26000EE926020EEA22EE52E55238
:1014B000E750EF6E040EE76E030EDBCFE9FF040E7C
:1014C000DBCFEAFFE750E926000EEA22030EEA022C
:1014D000F3CFEAFFE902F3CFE9FFF450EA26000E6A
:1014E000E926020EEA22EE52EF50E66EDF50EA6A7B
:1014F000590FE96E010EEA22EF50080BE66E6CEC14
:1015000001F0E552E552F350E66E040EE76E030E6D
:10151000DBCFE9FF040EDBCFEAFFE750E926000E40
:10152000EA22030EEA02F3CFEAFFE902F3CFE9FF72
:10153000F450EA26000EE926020EEA22EE52E552A7
:10154000E750EF6E050EE76E030EDBCFE9FF040EEA
:10155000DBCFEAFFE750E926000EEA22030EEA029B
:10156000F3CFEAFFE902F3CFE9FFF450EA26000ED9
:10157000E926020EEA22EE52EF50E66EDF50EA6AEA
:10158000590FE96E010EEA22EF50040BE66E6CEC87
:1015900001F0E552E552F350E66E050EE76E030EDC
:1015A000DBCFE9FF040EDBCFEAFFE750E926000EB0
:1015B000EA22030EEA02F3CFEAFFE902F3CFE9FFE2
:1015C000F450EA26000EE926020EEA22EE52E55217
:1015D000E750EF6E060EE76E030EDBCFE9FF040E59
:1015E000DBCFEAFFE750E926000EEA22030EEA020B
:1015F000F3CFEAFFE902F3CFE9FFF450EA26000E49
:10160000E926020EEA22EE52EF50E66EDF50EA6A59
:10161000590FE96E010EEA22EF50020BE66E6CECF8
:1016200001F0E552E552F350E66E060EE76E030E4A
:10163000DBCFE9FF040EDBCFEAFFE750E926000E1F
:10164000EA22030EEA02F3CFEAFFE902F3CFE9FF51
:10165000F450EA26000EE926020EEA22EE52E55286
:10166000E750EF6E070EE76E030EDBCFE9FF040EC7
:10167000DBCFEAFFE750E926000EEA22030EEA027A
:10168000F3CFEAFFE902F3CFE9FFF450EA26000EB8
:10169000E926020EEA22EE52EF50E66EDF50EA6AC9
:1016A000590FE96E010EEA22EF50010BE66E6CEC69
:1016B00001F0E552E552F350E66E070EE76E030EB9
:1016C000DBCFE9FF040EDBCFEAFFE750E926000E8F
:1016D000EA22030EEA02F3CFEAFFE902F3CFE9FFC1
:1016E000F450EA26000EE926020EEA22EE52E552F6
:1016F000E750EF6E030EDBCFE9FF040EDBCFEAFF0E
:10170000030EEA02F3CFEAFFE902F3CFE9FFF45058
:10171000EA26000EE926020EEA22020EE926000E53
:10172000EA22EF50E66EDF50EA6A610FE96E010EC1
:10173000EA22EF50800BE66E6CEC01F0E552E552C8
:10174000F350E66E030EDBCFE9FF040EDBCFEAFFBA
:10175000030EEA02F3CFEAFFE902F3CFE9FFF45008
:10176000EA26000EE926020EEA22020EE926000E03
:10177000EA22E552E750EF6E010EE76E030EDBCF73
:10178000E9FF040EDBCFEAFFE750E926000EEA226C
:10179000030EEA02F3CFEAFFE902F3CFE9FFF450C8
:1017A000EA26000EE926020EEA22020EE926000EC3
:1017B000EA22EF50E66EDF50EA6A610FE96E010E31
:1017C000EA22EF50400BE66E6CEC01F0E552E55278
:1017D000F350E66E010EE76E030EDBCFE9FF040E59
:1017E000DBCFEAFFE750E926000EEA22030EEA0209
:1017F000F3CFEAFFE902F3CFE9FFF450EA26000E47
:10180000E926020EEA22020EE926000EEA22E5523D
:10181000E750EF6E020EE76E030EDBCFE9FF040E1A
:10182000DBCFEAFFE750E926000EEA22030EEA02C8
:10183000F3CFEAFFE902F3CFE9FFF450EA26000E06
:10184000E926020EEA22020EE926000EEA22EF50F5
:10185000E66EDF50EA6A610FE96E010EEA22EF5090
:10186000200BE66E6CEC01F0E552E552F350E66EAB
:10187000020EE76E030EDBCFE9FF040EDBCFEAFFBB
:10188000E750E926000EEA22030EEA02F3CFEAFF50
:10189000E902F3CFE9FFF450EA26000EE926020E32
:1018A000EA22020EE926000EEA22E552E750EF6E28
:1018B000030EE76EDBCFE9FF040EDBCFEAFFE75054
:1018C000E926000EEA22030EEA02F3CFEAFFE9025C
:1018D000F3CFE9FFF450EA26000EE926020EEA22D1
:1018E000020EE926000EEA22EF50E66EDF50EA6AA9
:1018F000610FE96E010EEA22EF50100BE66E6CEC00
:1019000001F0E552E552F350E66E030EE76EDBCFD1
:10191000E9FF040EDBCFEAFFE750E926000EEA22DA
:10192000030EEA02F3CFEAFFE902F3CFE9FFF45036
:10193000EA26000EE926020EEA22020EE926000E31
:10194000EA22E552E750EF6E040EE76E030EDBCF9E
:10195000E9FF040EDBCFEAFFE750E926000EEA229A
:10196000030EEA02F3CFEAFFE902F3CFE9FFF450F6
:10197000EA26000EE926020EEA22020EE926000EF1
:10198000EA22EF50E66EDF50EA6A610FE96E010E5F
:10199000EA22EF50080BE66E6CEC01F0E552E552DE
:1019A000F350E66E040EE76E030EDBCFE9FF040E84
:1019B000DBCFEAFFE750E926000EEA22030EEA0237
:1019C000F3CFEAFFE902F3CFE9FFF450EA26000E75
:1019D000E926020EEA22020EE926000EEA22E5526C
:1019E000E750EF6E050EE76E030EDBCFE9FF040E46
:1019F000DBCFEAFFE750E926000EEA22030EEA02F7
:101A0000F3CFEAFFE902F3CFE9FFF450EA26000E34
:101A1000E926020EEA22020EE926000EEA22EF5023
:101A2000E66EDF50EA6A610FE96E010EEA22EF50BE
:101A3000040BE66E6CEC01F0E552E552F350E66EF5
:101A4000050EE76E030EDBCFE9FF040EDBCFEAFFE6
:101A5000E750E926000EEA22030EEA02F3CFEAFF7E
:101A6000E902F3CFE9FFF450EA26000EE926020E60
:101A7000EA22020EE926000EEA22E552E750EF6E56
:101A8000060EE76E030EDBCFE9FF040EDBCFEAFFA5
:101A9000E750E926000EEA22030EEA02F3CFEAFF3E
:101AA000E902F3CFE9FFF450EA26000EE926020E20
:101AB000EA22020EE926000EEA22EF50E66EDF501F
:101AC000EA6A610FE96E010EEA22EF50020BE66E40
:101AD0006CEC01F0E552E552F350E66E060EE76E4F
:101AE000030EDBCFE9FF040EDBCFEAFFE750E92668
:101AF000000EEA22030EEA02F3CFEAFFE902F3CF77
:101B0000E9FFF450EA26000EE926020EEA22020E50
:101B1000E926000EEA22E552E750EF6E070EE76E67
:101B2000030EDBCFE9FF040EDBCFEAFFE750E92627
:101B3000000EEA22030EEA02F3CFEAFFE902F3CF36
:101B4000E9FFF450EA26000EE926020EEA22020E10
:101B5000E926000EEA22EF50E66EDF50EA6A610FD6
:101B6000E96E010EEA22EF50010BE66E6CEC01F01B
:101B7000E552E552F350E66E070EE76E030EDBCF3B
:101B8000E9FF040EDBCFEAFFE750E926000EEA2268
:101B9000030EEA02F3CFEAFFE902F3CFE9FFF450C4
:101BA000EA26000EE926020EEA22020EE926000EBF
:101BB000EA22E552E750EF6EDF2A14EF07F0010149
:101BC000AA51B15D02E2B12901D0000EB16F79EFE7
:101BD00015F0B15101E0B9D0DF6A080EDF5C01E316
:101BE00085D0DF50EA6A510FE96E010EEA22EF6AF2
:101BF000DF50EA6A590FE96E010EEA22EF6ADF5000
:101C0000EA6A610FE96E010EEA22EF6A010EDB6AF1
:101C1000080EF36E010EDBCFF4FFF350F45C64E2C8
:101C20009AEC17F0F3CF14F0F4CF15F0040ED8901F
:101C300015321432E804FBE10001156A030E141694
:101C4000141801E115503BE0020E141801E1155083
:101C500026E0010E141801E1155004E0145041E192
:101C600015503FD0010EF36EDB5004E0D890F336F0
:101C7000E806FCE1F350146EDF50EA6A510FE96E9A
:101C8000010EEA22EF50F324E66EDF50EA6A510FAC
:101C9000E96E010EEA22E552E750EF6E22D0010E06
:101CA000F36EDB5004E0D890F336E806FCE1F35025
:101CB000146EDF50EA6A590FE96E010E0FD0010E63
:101CC000F36EDB5004E0D890F336E806FCE1F35005
:101CD000146EDF50EA6A610FE96E010EEA221450B9
:101CE000EF12010EDB2A94D7DF2A77D79AEC17F090
:101CF000F350DF6E0101ADC114F0AEC115F0AD2B94
:101D0000000EAE23166AACC1E9FFEA6AE9BEEA68D2
:101D1000030EEA02F3CFEAFFE902F3CFE9FFF45042
:101D2000EA266B0EE926010EEA22EE501424F36E29
:101D3000EE501520F46EEE501620F86EF4CFF7FF3B
:101D4000F3CFF6FF0800F5CFAAF1DF6A080EDF5CDB
:101D500002E371EF15F0080EDF02F350E66ED95082
:101D6000030FE96EDACFEAFFE552E750EE6EED6A57
:101D7000030EDBCFE9FF040EDBCFEAFF030EEA021E
:101D8000F3CFEAFFE902F3CFE9FFF450EA26000EB1
:101D9000E926020EEA22EF50E66EDF50EA6A510FA2
:101DA000E96E010EEA22EF50800BE66E6CEC01F05A
:101DB000E552E552F350E66E030EDBCFE9FF040E69
:101DC000DBCFEAFF030EEA02F3CFEAFFE902F3CF2B
:101DD000E9FFF450EA26000EE926020EEA22E55257
:101DE000E750EF6E010EE76E030EDBCFE9FF040E46
:101DF000DBCFEAFFE750E926000EEA22030EEA02F3
:101E0000F3CFEAFFE902F3CFE9FFF450EA26000E30
:101E1000E926020EEA22EF50E66EDF50EA6A510F21
:101E2000E96E010EEA22EF50400BE66E6CEC01F019
:101E3000E552E552F350E66E010EE76E030EDBCF7E
:101E4000E9FF040EDBCFEAFFE750E926000EEA22A5
:101E5000030EEA02F3CFEAFFE902F3CFE9FFF45001
:101E6000EA26000EE926020EEA22E552E750EF6E5E
:101E7000020EE76E030EDBCFE9FF040EDBCFEAFFB5
:101E8000E750E926000EEA22030EEA02F3CFEAFF4A
:101E9000E902F3CFE9FFF450EA26000EE926020E2C
:101EA000EA22EF50E66EDF50EA6A510FE96E010E4A
:101EB000EA22EF50200BE66E6CEC01F0E552E552A1
:101EC000F350E66E020EE76E030EDBCFE9FF040E61
:101ED000DBCFEAFFE750E926000EEA22030EEA0212
:101EE000F3CFEAFFE902F3CFE9FFF450EA26000E50
:101EF000E926020EEA22E552E750EF6E030EE76E86
:101F0000DBCFE9FF040EDBCFEAFFE750E926000E46
:101F1000EA22030EEA02F3CFEAFFE902F3CFE9FF78
:101F2000F450EA26000EE926020EEA22EF50E66E91
:101F3000DF50EA6A510FE96E010EEA22EF50100BF2
:101F4000E66E6CEC01F0E552E552F350E66E030EDE
:101F5000E76EDBCFE9FF040EDBCFEAFFE750E926AF
:101F6000000EEA22030EEA02F3CFEAFFE902F3CF02
:101F7000E9FFF450EA26000EE926020EEA22E552B5
:101F8000E750EF6E040EE76E030EDBCFE9FF040EA1
:101F9000DBCFEAFFE750E926000EEA22030EEA0251
:101FA000F3CFEAFFE902F3CFE9FFF450EA26000E8F
:101FB000E926020EEA22EF50E66EDF50EA6A510F80
:101FC000E96E010EEA22EF50080BE66E6CEC01F0B0
:101FD000E552E552F350E66E040EE76E030EDBCFDA
:101FE000E9FF040EDBCFEAFFE750E926000EEA2204
:101FF000030EEA02F3CFEAFFE902F3CFE9FFF45060
:10200000EA26000EE926020EEA22E552E750EF6EBC
:10201000050EE76E030EDBCFE9FF040EDBCFEAFF10
:10202000E750E926000EEA22030EEA02F3CFEAFFA8
:10203000E902F3CFE9FFF450EA26000EE926020E8A
:10204000EA22EF50E66EDF50EA6A510FE96E010EA8
:10205000EA22EF50040BE66E6CEC01F0E552E5521B
:10206000F350E66E050EE76E030EDBCFE9FF040EBC
:10207000DBCFEAFFE750E926000EEA22030EEA0270
:10208000F3CFEAFFE902F3CFE9FFF450EA26000EAE
:10209000E926020EEA22E552E750EF6E060EE76EE1
:1020A000030EDBCFE9FF040EDBCFEAFFE750E926A2
:1020B000000EEA22030EEA02F3CFEAFFE902F3CFB1
:1020C000E9FFF450EA26000EE926020EEA22EF505C
:1020D000E66EDF50EA6A510FE96E010EEA22EF5018
:1020E000020BE66E6CEC01F0E552E552F350E66E41
:1020F000060EE76E030EDBCFE9FF040EDBCFEAFF2F
:10210000E750E926000EEA22030EEA02F3CFEAFFC7
:10211000E902F3CFE9FFF450EA26000EE926020EA9
:10212000EA22E552E750EF6E070EE76E030EDBCFB3
:10213000E9FF040EDBCFEAFFE750E926000EEA22B2
:10214000030EEA02F3CFEAFFE902F3CFE9FFF4500E
:10215000EA26000EE926020EEA22EF50E66EDF5074
:10216000EA6A510FE96E010EEA22EF50010BE66EAA
:102170006CEC01F0E552E552F350E66E070EE76EA7
:10218000030EDBCFE9FF040EDBCFEAFFE750E926C1
:10219000000EEA22030EEA02F3CFEAFFE902F3CFD0
:1021A000E9FFF450EA26000EE926020EEA22E55283
:1021B000E750EF6E030EDBCFE9FF040EDBCFEAFF43
:1021C000030EEA02F3CFEAFFE902F3CFE9FFF4508E
:1021D000EA26000EE926020EEA22EE52EF50E66EE3
:1021E000DF50EA6A590FE96E010EEA22EF50800BC8
:1021F000E66E6CEC01F0E552E552F350E66E030E2C
:10220000DBCFE9FF040EDBCFEAFF030EEA02F3CFD8
:10221000EAFFE902F3CFE9FFF450EA26000EE926CF
:10222000020EEA22EE52E552E750EF6E010EE76E23
:10223000030EDBCFE9FF040EDBCFEAFFE750E92610
:10224000000EEA22030EEA02F3CFEAFFE902F3CF1F
:10225000E9FFF450EA26000EE926020EEA22EE52C9
:10226000EF50E66EDF50EA6A590FE96E010EEA227E
:10227000EF50400BE66E6CEC01F0E552E552F35086
:10228000E66E010EE76E030EDBCFE9FF040EDBCF37
:10229000EAFFE750E926000EEA22030EEA02F3CF36
:1022A000EAFFE902F3CFE9FFF450EA26000EE9263F
:1022B000020EEA22EE52E552E750EF6E020EE76E92
:1022C000030EDBCFE9FF040EDBCFEAFFE750E92680
:1022D000000EEA22030EEA02F3CFEAFFE902F3CF8F
:1022E000E9FFF450EA26000EE926020EEA22EE5239
:1022F000EF50E66EDF50EA6A590FE96E010EEA22EE
:10230000EF50200BE66E6CEC01F0E552E552F35015
:10231000E66E020EE76E030EDBCFE9FF040EDBCFA5
:10232000EAFFE750E926000EEA22030EEA02F3CFA5
:10233000EAFFE902F3CFE9FFF450EA26000EE926AE
:10234000020EEA22EE52E552E750EF6E030EE76E00
:10235000DBCFE9FF040EDBCFEAFFE750E926000EF2
:10236000EA22030EEA02F3CFEAFFE902F3CFE9FF24
:10237000F450EA26000EE926020EEA22EE52EF5051
:10238000E66EDF50EA6A590FE96E010EEA22EF505D
:10239000100BE66E6CEC01F0E552E552F350E66E80
:1023A000030EE76EDBCFE9FF040EDBCFEAFFE75059
:1023B000E926000EEA22030EEA02F3CFEAFFE90261
:1023C000F3CFE9FFF450EA26000EE926020EEA22D6
:1023D000EE52E552E750EF6E040EE76E030EDBCFD0
:1023E000E9FF040EDBCFEAFFE750E926000EEA2200
:1023F000030EEA02F3CFEAFFE902F3CFE9FFF4505C
:10240000EA26000EE926020EEA22EE52EF50E66EB0
:10241000DF50EA6A590FE96E010EEA22EF50080B0D
:10242000E66E6CEC01F0E552E552F350E66E040EF8
:10243000E76E030EDBCFE9FF040EDBCFEAFFE750C8
:10244000E926000EEA22030EEA02F3CFEAFFE902D0
:10245000F3CFE9FFF450EA26000EE926020EEA2245
:10246000EE52E552E750EF6E050EE76E030EDBCF3E
:10247000E9FF040EDBCFEAFFE750E926000EEA226F
:10248000030EEA02F3CFEAFFE902F3CFE9FFF450CB
:10249000EA26000EE926020EEA22EE52EF50E66E20
:1024A000DF50EA6A590FE96E010EEA22EF50040B81
:1024B000E66E6CEC01F0E552E552F350E66E050E67
:1024C000E76E030EDBCFE9FF040EDBCFEAFFE75038
:1024D000E926000EEA22030EEA02F3CFEAFFE90240
:1024E000F3CFE9FFF450EA26000EE926020EEA22B5
:1024F000EE52E552E750EF6E060EE76E030EDBCFAD
:10250000E9FF040EDBCFEAFFE750E926000EEA22DE
:10251000030EEA02F3CFEAFFE902F3CFE9FFF4503A
:10252000EA26000EE926020EEA22EE52EF50E66E8F
:10253000DF50EA6A590FE96E010EEA22EF50020BF2
:10254000E66E6CEC01F0E552E552F350E66E060ED5
:10255000E76E030EDBCFE9FF040EDBCFEAFFE750A7
:10256000E926000EEA22030EEA02F3CFEAFFE902AF
:10257000F3CFE9FFF450EA26000EE926020EEA2224
:10258000EE52E552E750EF6E070EE76E030EDBCF1B
:10259000E9FF040EDBCFEAFFE750E926000EEA224E
:1025A000030EEA02F3CFEAFFE902F3CFE9FFF450AA
:1025B000EA26000EE926020EEA22EE52EF50E66EFF
:1025C000DF50EA6A590FE96E010EEA22EF50010B63
:1025D000E66E6CEC01F0E552E552F350E66E070E44
:1025E000E76E030EDBCFE9FF040EDBCFEAFFE75017
:1025F000E926000EEA22030EEA02F3CFEAFFE9021F
:10260000F3CFE9FFF450EA26000EE926020EEA2293
:10261000EE52E552E750EF6E030EDBCFE9FF040EFA
:10262000DBCFEAFF030EEA02F3CFEAFFE902F3CFC2
:10263000E9FFF450EA26000EE926020EEA22020E15
:10264000E926000EEA22EF50E66EDF50EA6A610FDB
:10265000E96E010EEA22EF50800BE66E6CEC01F0A1
:10266000E552E552F350E66E030EDBCFE9FF040EB0
:10267000DBCFEAFF030EEA02F3CFEAFFE902F3CF72
:10268000E9FFF450EA26000EE926020EEA22020EC5
:10269000E926000EEA22E552E750EF6E010EE76EE2
:1026A000030EDBCFE9FF040EDBCFEAFFE750E9269C
:1026B000000EEA22030EEA02F3CFEAFFE902F3CFAB
:1026C000E9FFF450EA26000EE926020EEA22020E85
:1026D000E926000EEA22EF50E66EDF50EA6A610F4B
:1026E000E96E010EEA22EF50400BE66E6CEC01F051
:1026F000E552E552F350E66E010EE76E030EDBCFB6
:10270000E9FF040EDBCFEAFFE750E926000EEA22DC
:10271000030EEA02F3CFEAFFE902F3CFE9FFF45038
:10272000EA26000EE926020EEA22020EE926000E33
:10273000EA22E552E750EF6E020EE76E030EDBCFA2
:10274000E9FF040EDBCFEAFFE750E926000EEA229C
:10275000030EEA02F3CFEAFFE902F3CFE9FFF450F8
:10276000EA26000EE926020EEA22020EE926000EF3
:10277000EA22EF50E66EDF50EA6A610FE96E010E61
:10278000EA22EF50200BE66E6CEC01F0E552E552C8
:10279000F350E66E020EE76E030EDBCFE9FF040E88
:1027A000DBCFEAFFE750E926000EEA22030EEA0239
:1027B000F3CFEAFFE902F3CFE9FFF450EA26000E77
:1027C000E926020EEA22020EE926000EEA22E5526E
:1027D000E750EF6E030EE76EDBCFE9FF040EDBCFB1
:1027E000EAFFE750E926000EEA22030EEA02F3CFE1
:1027F000EAFFE902F3CFE9FFF450EA26000EE926EA
:10280000020EEA22020EE926000EEA22EF50E66EE0
:10281000DF50EA6A610FE96E010EEA22EF50100BF9
:10282000E66E6CEC01F0E552E552F350E66E030EF5
:10283000E76EDBCFE9FF040EDBCFEAFFE750E926C6
:10284000000EEA22030EEA02F3CFEAFFE902F3CF19
:10285000E9FFF450EA26000EE926020EEA22020EF3
:10286000E926000EEA22E552E750EF6E040EE76E0D
:10287000030EDBCFE9FF040EDBCFEAFFE750E926CA
:10288000000EEA22030EEA02F3CFEAFFE902F3CFD9
:10289000E9FFF450EA26000EE926020EEA22020EB3
:1028A000E926000EEA22EF50E66EDF50EA6A610F79
:1028B000E96E010EEA22EF50080BE66E6CEC01F0B7
:1028C000E552E552F350E66E040EE76E030EDBCFE1
:1028D000E9FF040EDBCFEAFFE750E926000EEA220B
:1028E000030EEA02F3CFEAFFE902F3CFE9FFF45067
:1028F000EA26000EE926020EEA22020EE926000E62
:10290000EA22E552E750EF6E050EE76E030EDBCFCD
:10291000E9FF040EDBCFEAFFE750E926000EEA22CA
:10292000030EEA02F3CFEAFFE902F3CFE9FFF45026
:10293000EA26000EE926020EEA22020EE926000E21
:10294000EA22EF50E66EDF50EA6A610FE96E010E8F
:10295000EA22EF50040BE66E6CEC01F0E552E55212
:10296000F350E66E050EE76E030EDBCFE9FF040EB3
:10297000DBCFEAFFE750E926000EEA22030EEA0267
:10298000F3CFEAFFE902F3CFE9FFF450EA26000EA5
:10299000E926020EEA22020EE926000EEA22E5529C
:1029A000E750EF6E060EE76E030EDBCFE9FF040E75
:1029B000DBCFEAFFE750E926000EEA22030EEA0227
:1029C000F3CFEAFFE902F3CFE9FFF450EA26000E65
:1029D000E926020EEA22020EE926000EEA22EF5054
:1029E000E66EDF50EA6A610FE96E010EEA22EF50EF
:1029F000020BE66E6CEC01F0E552E552F350E66E28
:102A0000060EE76E030EDBCFE9FF040EDBCFEAFF15
:102A1000E750E926000EEA22030EEA02F3CFEAFFAE
:102A2000E902F3CFE9FFF450EA26000EE926020E90
:102A3000EA22020EE926000EEA22E552E750EF6E86
:102A4000070EE76E030EDBCFE9FF040EDBCFEAFFD4
:102A5000E750E926000EEA22030EEA02F3CFEAFF6E
:102A6000E902F3CFE9FFF450EA26000EE926020E50
:102A7000EA22020EE926000EEA22EF50E66EDF504F
:102A8000EA6A610FE96E010EEA22EF50010BE66E71
:102A90006CEC01F0E552E552F350E66E070EE76E7E
:102AA000030EDBCFE9FF040EDBCFEAFFE750E92698
:102AB000000EEA22030EEA02F3CFEAFFE902F3CFA7
:102AC000E9FFF450EA26000EE926020EEA22020E81
:102AD000E926000EEA22E552E750EF6EDF2AA6EF64
:102AE0000EF00101AA51B15D02E2B12901D0000E40
:102AF000B16F4F0E166E580E176E000E186EACC1E9
:102B000019F01A6A1B6A19AE02D01A681B68D890AD
:102B100019361A361B3616501924F36E17501A2020
:102B2000F46E18501B20F86EF4CFF7FFF3CFF6FFCA
:102B30000900F5CF14F00800F5CF15F0010114508D
:102B4000AD5D1550AE5915E3AD6BAE6B010150058F
:102B5000506F0101A70502E0000E01D0010E146EB6
:102B60000101505102E0000E01D0010E141401E0E9
:102B700037D9050EE15C02E2E16AE552E16EE55209
:102B8000E7CFD9FF1200D9CFE6FFE1CFD9FF020E80
:102B9000E1260101B05156E1DF6A040EDF5C48E234
:102BA000DF50030DF3CFE9FFF4CFEAFF000EE92673
:102BB000020EEA22EECF14F0EECF15F0EFCF16F0B2
:102BC000DF50030DF3CFE9FFF4CFEAFFC00EE92693
:102BD000020EEA2214C0EEFF15C0EEFF16C0EEFF93
:102BE000DF50030DF3CFE9FFF4CFEAFF000EE92633
:102BF000020EEA22EF6ADF50030DF3CFE9FFF4CFB4
:102C0000EAFF000EE926020EEA22EE52EF6ADF50DA
:102C1000030DF3CFE9FFF4CFEAFF000EE926020E21
:102C2000EA22020EE926000EEA22EF6ADF2AB5D771
:102C300060C2CCF261C2CDF262C2CEF20201606B20
:102C4000616B626B0101AC29E76E010EE7CFDBFF20
:102C5000A75102E0FF0E01D0000E0201626F010ECB
:102C6000DB50010B02E0FF0E01D0000E006F010EE1
:102C7000DB50020B02E0FF0E01D0000E036F010ECD
:102C8000DB50040B02E0FF0E01D0000E066F010EB8
:102C9000DB50080B02E0FF0E01D0000E096F0101AE
:102CA000B02B9288928A8050200B200A01E0010EFE
:102CB000146E8050100B100A01E0010E141417E07E
:102CC000B051400801E382D0A75102E0000E01D0CC
:102CD000010EA76F07EC00F0A7C1E6FF000EE66E3D
:102CE000E66A95EC36F0E552E552E5520DD080B833
:102CF00005D0B05140086AE273D806D080BA08D037
:102D0000B051400863E2C1D80101010EB06F5ED03E
:102D1000DF6ADF50DF2A000927E0DF50030DF3CF21
:102D2000E9FFF4CFEAFFC00EE926020EEA22EECF59
:102D300014F0EECF15F0EFCF16F0DF50030DF3CF08
:102D4000E9FFF4CFEAFF000EE926020EEA2214C0E2
:102D5000EEFF15C0EEFF16C0EEFF040EDF5C02E3CF
:102D6000000ED7D7010ED5D7CCC260F2CDC261F22A
:102D7000CEC262F20101B06BA7C114F0156A14BE95
:102D8000156814C0E6FF15C0E6FFACC116F0176A5F
:102D900016BE176816C0E6FF17C0E6FF700EE66E97
:102DA0006C0EE66E000EE66E000EE66E010EE66E2E
:102DB000E8EC34F0186E090EE15E1850000EE66E75
:102DC000010EE66E57EC32F0E552E552020EE15C80
:102DD00002E2E16AE552E16EE552E7CFD9FF120067
:102DE0000E0E0101E76EAC19E8AE02D0E73402D056
:102DF000E750AC5D02E3000E01D0AC29AC6FAD6BC7
:102E0000AE6B6D0E146E580E156E000E166EACC1C4
:102E100017F0186A196A17AE02D0186819681450AA
:102E20001724F36E15501820F46E16501920F86E02
:102E3000F4CFF7FFF3CFF6FF0800F5CF50F1010113
:102E40005051E66EE66AACC114F0156A14BE1568FE
:102E500014C0E6FF15C0E6FF5C0EE66E6C0EE66E73
:102E6000000EE66E000EE66E010EE66EE8EC34F043
:102E7000166E090EE15E1650000EE66E010EE66E4D
:102E800057EC32F0E552E5521200010E0101E76EF7
:102E9000AC19E8AE02D0E73402D0E750AC5D02E2F4
:102EA0000E0E01D0AC05AC6FAD6BAE6B6D0E146E3B
:102EB000580E156E000E166EACC117F0186A196A1E
:102EC00017AE02D01868196814501724F36E155005
:102ED0001820F46E16501920F86EF4CFF7FFF3CFD8
:102EE000F6FF0800F5CF50F101015051E66EE66A99
:102EF000ACC114F0156A14BE156814C0E6FF15C005
:102F0000E6FF460EE66E6C0EE66E000EE66E000EF6
:102F1000E66E010EE66EE8EC34F0166E090EE15E28
:102F20001650000EE66E010EE66E57EC32F0E552DA
:102F3000E5521200D9CFE6FFE1CFD9FF020EE1261C
:102F4000B2C11AF0B3C11BF0D8901B321A32D8901C
:102F50001B321A320101B2511A18186EB3511B18E4
:102F6000196EB2C11CF0B3C11DF0030ED8901D3212
:102F70001C32E804FBE118501C18166E19501D187D
:102F8000176EB2C11EF0B3C11FF0050ED8901F32EC
:102F90001E32E804FBE116501E18146E17501F185D
:102FA000156E010E1416000E151614C0DEFF15C0A6
:102FB000DDFFB2C114F0B3C115F0D8901532143250
:102FC000DECF16F0DDCF17F01640166A800B176EB5
:102FD000145016100101B26F15501710B36FB2C123
:102FE000F3FFF46E020EE15C02E2E16AE552E16E8B
:102FF000E552E7CFD9FF1200D9CFE6FFE1CFD9FFE5
:10300000020EE126B59EB588B59C8F0ED3147009CB
:10301000D36E0F0EC16E300E926E936A946A806A00
:10302000816A826AC2D875EC1AF0949E938093925A
:103030009396939492909292929492969398939A54
:10304000939C939E89908992899489968A988A9A6A
:103050008A9C8A9E8A968A94E66AE66AE66AC8EC40
:1030600036F0E552E552E552070EB16EB46A010E34
:10307000DB6A400EF36E010EDBCFF4FFF350F45C1D
:103080002DE2010EDB50030DF3CFE9FFF4CFEAFF91
:10309000000EE926020EEA22070EEF6E010EDB504B
:1030A000030DF3CFE9FFF4CFEAFF000EE926020E8D
:1030B000EA22EE52EF6A010EDB50030DF3CFE9FF77
:1030C000F4CFEAFF000EE926020EEA22020EE926FC
:1030D000000EEA22EF6A010EDB2ACBD7D08ED09CFD
:1030E000A282B180A082F28EF19E0F015B6B856A95
:1030F000020EE15C02E2E16AE552E16EE552E7CFE1
:10310000D9FF1200D9CFE6FFE1CFD9FFFD0EDBCF0B
:10311000E6FF5EEC37F0E552FE0EDBCFE6FF5EEC3D
:1031200037F0E552FB0EDB500101B45D09E08990F8
:103130008992899489968A988A9A8A9C8A9E89908B
:10314000FC0EDBCFE6FF5EEC37F0E5528A848A9412
:10315000FB0EDB500101B45D21E0FB0EDB50070AE2
:103160001CE0010A18E0030A14E0010A10E0070A53
:103170000CE0010A08E0030A04E0010A0FE189807B
:103180000DD089820BD0898409D0898607D08A889E
:1031900005D08A8A03D08A8C01D08A8EFB0EDBCFC1
:1031A000B4F1E552E7CFD9FF1200400E8B1694160A
:1031B0009288928A01019F6BA06BA16BA26B120097
:1031C000200E0201E76ECF19E8AE02D0E73402D03C
:1031D000E750CF5D01E2FCD06050020B01E012002D
:1031E00001019F51A01102E1000E08D09FC1E9FF2B
:1031F000A0C1EAFFEF50800B01E0010E000901E0E1
:10320000E7D005010051840A01E1C8D0070A01E1B5
:103210009BD0010A70E0030A51E0010A1DE0900A08
:1032200001E0C3D0400EE66E050EE66E14EC33F0FE
:10323000E552E5520101A151A21102E1000E08D0B0
:10324000A1C1E9FFA2C1EAFFEF50800B01E0010E2E
:10325000000901E0AAD064D001019C51E66EE66A43
:10326000380EE66E6C0EE66E000EE66E000EE66E32
:10327000010EE66EE8EC34F0146E070EE15E1450B9
:10328000000EE66E010EE66E57EC32F0E552E552A6
:103290008B7C010EE66E0F0EE66EAA0EE66E550EE4
:1032A000E66E30DFE552E552E552E5520101A651E6
:1032B00002E0000E01D0010EA66F77D08050200BE7
:1032C00001E0010EE824146E8050100B01E0010EA5
:1032D0001424406F0101A151A21102E1000E08D097
:1032E000A1C1E9FFA2C1EAFFEF50800B01E0010E8E
:1032F00000095BE115D08B50400B01E0010E406FDF
:103300000101A151A21102E1000E08D0A1C1E9FF03
:10331000A2C1EAFFEF50800B01E0010E000945E178
:10332000400EE66E400EE66E050EE66E010EE66E8F
:10333000E66EEBEC1BF0146E050EE15E1450F3CF5D
:10334000A1F1F4CFA2F131D00451030DF3CFE9FF85
:10335000F4CFEAFF000EE926020EEA2201C5EFFFD4
:103360000451030DF3CFE9FFF4CFEAFF000EE92685
:10337000020EEA22EE5202C5EFFF0451030DF3CF15
:10338000E9FFF4CFEAFF000EE926020EEA22020E60
:10339000E926000EEA2203C5EFFF07D0015102E142
:1033A0001FDD03D0010501E170DD400EE66E000E69
:1033B000E66E050EE66EE66A010EE66EEBEC1BF0BD
:1033C000146E050EE15E1450F3CF9FF1F4CFA0F11F
:1033D0001200120012001200120027EF34F0120047
:1033E0001E0EE66E010EE66EB4EC1BF0E552E552E1
:1033F000400EE66E000EE66E050EE66EE66A010E03
:10340000E66EEBEC1BF0146E050EE15E1450F3CF8C
:103410009FF1F4CFA0F112000201F00520E10201BA
:10342000F1051DE1A394D6DF60920201F16B010169
:10343000100E696F0E0E6A6F6907000E6A5B6951A4
:103440006A11FAE16084080E696F070E6A6F6907F6
:10345000000E6A5B69516A11FAE16094A38412005C
:10346000D9CFE6FFE1CFD9FFFD0EDBCF08F0FE0E8E
:10347000DBCF09F0E868081802E17F0E09182FE099
:10348000030E081801E1095028E0020E081801E1B6
:10349000095021E0010E081801E109501AE0740EEC
:1034A000081801E1095013E0750E081801E10950F0
:1034B0000CE0730E081801E1095005E0720E0818BF
:1034C0000FE109500DD087DF0BD083DF09D082DFF9
:1034D00007D086DF05D083DF03D07FDF01D07CDF1C
:0A34E000010EE552E7CFD9FF1200FC
:0634EA00D9CFE6FFE1CF9F
:1034F000D9FFE652A394676A656A6A6A010EE66EAE
:10350000E66AE66A6B0EE66E0F0EE66E8DEC35F03F
:10351000146E050EE15E1450160E626E9F0E666EFE
:103520007B0E646EDF6ADF50146E156A080E145C41
:10353000000E155810E2DF50040DF3CFE9FFF4CF71
:10354000EAFF000EE926040EEA22EE6AEE6AEE6A4F
:10355000EE6ADF2AE8D7608C636A6098609C65A693
:1035600007D065960201E36BE86BE96BEA6BF7D76E
:103570000201010EFB6FFC6FFD6BFE6BF16BDF6AEE
:10358000020EDF5C26E2EA6ADF34FE0BEA36E96E01
:10359000DA0EE926020EEA22EE6AED6AEA6ADF3402
:1035A000FE0BEA36E96ED60EE926020EEA22EE6A34
:1035B000ED6ADF50EA6AF50FE96E020EEA22EF6A61
:1035C000DF50EA6AF70FE96E020EEA22EF6ADF2A9D
:1035D000D7D70201080EDA6F040EDB6F160E6A6E83
:1035E0000401200E026F040E036F080E016F840E9B
:1035F000006F0201D06BCF6BE552E552E7CFD9FFE8
:103600001200D9CFE6FFE1CFD9FFE6520201CF0584
:1036100007E160BA05D0656A64806488020ECF6FE6
:103620006550040B06E06450040B03E0659434EC31
:1036300021F060B259D06550010B09E06450010BD4
:1036400006E053DFA3840201040ECF6F659065503E
:10365000100B06E06450100B03E01FEC21F065989E
:1036600065AC19D064AC0FD0010EE66EE66A000EB0
:10367000E66EE66A730EE66EE66A30EC1AF0146ED9
:10368000060EE15E1450659C0201F95101E0F90754
:10369000F95101E1FBD96550200B05E06450200B86
:1036A00002E006EC21F06550020B13E06450020BBF
:1036B00010E0010EE66EE66A000EE66EE66AE66867
:1036C0007F0EE66E30EC1AF0146E060EE15E1450BA
:1036D000676A040E0201E76ECF19E8AE02D0E73444
:1036E00002D0E750CF5D02E2A49439D064A636D070
:1036F000DF6A040EDF5C32E265A630D061CFF2F201
:103700000201F251780BE842E842E842F36F659615
:10371000F2B506D0F351EA6AF70FE96E020E05D052
:10372000F351EA6AF50FE96E020EEA22EF70F351E7
:1037300003E14BEC21F010D0000EE66EE66AF20ECB
:10374000E66E020EE66E720EE66EE66A30EC1AF077
:10375000146E060EE15E1450DF2ACBD7A494E55216
:10376000E552E7CFD9FF1200D9CFE6FFE1CFD9FF6D
:10377000020EE126FD0EDBA407D0E66AFE0EDBCFCB
:10378000E6FF13DAE552E552FD0EDBA208D0010E8A
:10379000E66EFE0EDBCFE6FF08DAE552E552FE0EDE
:1037A000DB50156A6A0F146E0F0E152214C0DEFF6F
:1037B00015C0DDFFDECFE9FFDDCFEAFFFD0EDBCF79
:1037C000EFFF020EE15C02E2E16AE552E16EE552D2
:1037D000E7CFD9FF1200D9CFE6FFE1CFD9FF020E24
:1037E000E126FD0EDB500AE0FE0EEA6ADB34FE0B3A
:1037F000EA36E96EDA0EE926020E09D0FE0EEA6A12
:10380000DB34FE0BEA36E96ED60EE926020EEA221A
:10381000EECFDEFFEDCFDDFFD9CFE9FFDACFEAFF54
:10382000EE50ED1003E1F36AF46A44D0DECFE9FF15
:10383000DDCFEAFF020EE926000EEA22FB0EDBCF07
:10384000EEFFFC0EDBCFEDFFDECFE9FFDDCFEAFFC1
:10385000EE52FA0EDBCFEFFF400EDECFE9FFDDCFF9
:10386000EAFFE850EF16880EDECFE9FFDDCFEAFF72
:10387000E850EF12FD0EDB500AE0FE0EEA6ADB3480
:10388000FE0BEA36E96EDA0EE926020E09D0FE0ECC
:10389000EA6ADB34FE0BEA36E96ED60EE926020E42
:1038A000EA22EF74DECF14F0DDCF15F014C0F3FF81
:1038B00015C0F4FF020EE15C02E2E16AE552E16E3E
:1038C000E552E7CFD9FF1200D9CFE6FFE1CFD9FF0C
:1038D000020EE126FE0EDB5020E1D4C2E9FFD5C284
:1038E000EAFFEE52080EEF6ED4C2E9FFD5C2EAFF3E
:1038F000020EE926000EEA22200EEE6E040EED6E98
:10390000D4C2E9FFD5C2EAFF8C0EEF6EDAC2E9FF3E
:10391000DBC2EAFF840EEF6E3BD0FD0EDB50E824E5
:10392000166EFE0EDB50040DF3501624040DF3CF7B
:1039300014F0F4CF15F0000E1426040E152214C056
:10394000DEFF15C0DDFF840EDECFE9FFDDCFEAFF2D
:10395000E850EF12FD0EDB50E824166EFE0EDB5031
:10396000040DF3501624010F040DF3CF14F0F4CF1F
:1039700015F0000E1426040E152214C0DEFF15C02B
:10398000DDFF840EDECFE9FFDDCFEAFFE850EF1266
:10399000020EE15C02E2E16AE552E16EE552E7CF38
:1039A000D9FF1200D9CFE6FFE1CFD9FF60A84ED0F2
:1039B000FE0EEA6ADB34FE0BEA36E96EDA0EE92621
:1039C000020EEA22EE50EFCFEAFFE96E400EEE164D
:1039D000EE6AEE6AEE6AFE0EEA6ADB34FE0BEA3647
:1039E000E96EDA0EE926020EEA22EE50EFCFEAFF88
:1039F000E96EEE7CFE0EEA6ADB34FE0BEA36E96E17
:103A0000DA0EE926020EEA22EF74400E146EFE0E64
:103A1000EA6ADB34FE0BEA36E96EDA0EE926020EBC
:103A2000EA22EE50EFCFEAFFE96E1450EF16FE0ED9
:103A3000EA6ADB34FE0BEA36E96EDA0EE926020E9C
:103A4000EA22EE50EFCFEAFFE96EEF7CE552E7CFD6
:103A5000D9FF1200606A646A0201CF6B1200020192
:103A6000CF5113E1606A646A160E626E9F0E666E35
:103A70007B0E646ED08EA584A384F28E60B602D0D5
:103A80006086FCD70201010ECF6F12000201FB51CC
:103A90004DE1010EFB6FFC5149E1010EFC6F020E7E
:103AA000DF5D0DE1DAC2E9FFDBC2EAFFEE52EF6A49
:103AB000DAC2E9FFDBC2EAFFC80EEF6E1200DF05D3
:103AC00035E1F46BD2C2E9FFD3C2EAFFEE52080E31
:103AD000EF6ED2C2E9FFD3C2EAFF020EE926000E62
:103AE000EA22200EEE6E040EED6ED2C2E9FFD3C2C2
:103AF000EAFF840EEF6E010EF46FD4C2E9FFD5C267
:103B0000EAFFEE52080EEF6ED4C2E9FFD5C2EAFF1B
:103B1000020EE926000EEA22200EEE6E040EED6E75
:103B2000D4C2E9FFD5C2EAFF800EEF6E1200020197
:103B3000FD6BFE6B020EDF5D18E1D4C2E9FFD5C25A
:103B4000EAFFEE52080EEF6ED4C2E9FFD5C2EAFFDB
:103B5000020EE926000EEA22280EEE6E040EED6E2D
:103B6000D4C2E9FFD5C2EAFF1DD0E4510401265DAD
:103B70000201E5510401275904E226C4E4F227C4F6
:103B8000E5F2CAD8DAC2E9FFDBC2EAFF020EE92693
:103B9000000EEA22280EEE6E040EED6EDAC2E9FF88
:103BA000DBC2EAFFC80EEF6E1200D9CFE6FFE1CF0D
:103BB000D9FF020EE126000EDE6E040EDD6EFD0E54
:103BC000DB50E824166EFE0EDB50040DF350162475
:103BD000040DF4CF15F0D9CFE9FFDACFEAFFF350A7
:103BE000EE261550ED22DECFE9FFDDCFEAFFEF9E96
:103BF000FD0EDB500AE1FE0EEA6ADB34FE0BEA360C
:103C0000E96ED60EE926020E09D0FE0EEA6ADB3412
:103C1000FE0BEA36E96EDA0EE926020EEA22DECF64
:103C2000EEFFDDCFEDFFDECFE9FFDDCFEAFFEF9C5A
:103C3000DECFE9FFDDCFEAFF040EE926000EEA221F
:103C4000EF8C020EE15C02E2E16AE552E16EE552C0
:103C5000E7CFD9FF120060980201E3BF2BD0E8AF95
:103C600009D0020EDF6FFE5101E161DF0201FC6B42
:103C7000FB6B1200D4C2E9FFD5C2EAFFEE52080E78
:103C8000EF6ED4C2E9FFD5C2EAFF020EE926000EAC
:103C9000EA22200EEE6E040EED6ED4C2E9FFD5C20C
:103CA000EAFF8C0EEF6EDAC2E9FFDBC2EAFF840E98
:103CB000EF6E1200040120AF0DD00201010EDF6F84
:103CC000FD5101E134DF0201FC6BFB6BFA5123E192
:103CD00046EF1DF00201020EDF6FD4C2E9FFD5C22C
:103CE000EAFFEE52080EEF6ED4C2E9FFD5C2EAFF3A
:103CF000020EE926000EEA22200EEE6E040EED6E94
:103D0000D4C2E9FFD5C2EAFF840EEF6EFC6BFB6BF9
:103D1000FA5101E1BBDE1200D9CFE6FFE1CFD9FFB6
:103D2000E652080EDF6E0201E45D000EE5590AE27C
:103D3000E4C2DFFFDE5102E1010E03D0DE0502E145
:103D4000020EDE6FDF50156AE850E45DE46F155037
:103D5000E559E56FDAC2E9FFDBC2EAFFEE52DFCFD9
:103D6000EFFF280EEE6F040EEF6FE3B11BD0DF50B4
:103D700030E0E0C2F6FFE02BE1C2F7FF000EE123E6
:103D8000E2C2F8FFE2230800F550E66EEEC2E9FF5A
:103D9000EFC2EAFFEE2B000EEF23E552E750EF6E85
:103DA000DF06E5D7DF5015E0E0C2E9FFE1C2EAFF38
:103DB000E02B000EE123EF50E66EEEC2E9FFEFC20A
:103DC000EAFFEE2B000EEF23E552E750EF6EDF0621
:103DD000E9D7E552E552E7CFD9FF1200D9CFE6FF88
:103DE000E1CFD9FF020EE126D2C2E9FFD3C2EAFF3A
:103DF000EE52EFCFDFFFDFCF14F014500201E95D88
:103E0000000EEA5902E2E9C2DFFFDF50146E156AC4
:103E1000E850E95DE96F1550EA59EA6F010EDB6A77
:103E2000DF50F36E010EDBCFF4FFF350F45C16E2CB
:103E3000010EDB50EA6A280FE96E040EEA22EF5009
:103E4000E66EE6C2E9FFE7C2EAFFE62B000EE723D3
:103E5000E552E750EF6E010EDB2AE2D7000ED88064
:103E6000E955000EEA5527E2D4C2E9FFD5C2EAFFC0
:103E7000EE52080EEF6ED4C2E9FFD5C2EAFF020E81
:103E8000E926000EEA22280EEE6E040EED6ED2C276
:103E9000E9FFD3C2EAFFEF50400B06E1D4C2E9FFCD
:103EA000D5C2EAFFC80E05D0D4C2E9FFD5C2EAFFE9
:103EB000880EEF6E2BD0D4C2E9FFD5C2EAFFEE52D6
:103EC000080EEF6ED4C2E9FFD5C2EAFF020EE92662
:103ED000000EEA22200EEE6E040EED6ED4C2E9FF53
:103EE000D5C2EAFF840EEF6EEB51EC11ED1109E043
:103EF00007D0EDC2FBFFECC2FAFF0201EB51F96EF5
:103F0000F8DF0201E89FFA5101E1C0DD020EE15C39
:103F100002E2E16AE552E16EE552E7CFD9FF120015
:103F2000D9CFE6FFE1CFD9FFE6520201E38F010EC0
:103F3000E66EE66AE66A6B0EE66E0F0EE66E8DECD6
:103F400035F0146E050EE15E1450200EE66EE66A42
:103F5000E66A000EE66E040EE66E8DEC35F0146E29
:103F6000050EE15E1450608CDF6A020EDF5C10E229
:103F7000DF50EA6AF50FE96E020EEA22EF6ADF50BF
:103F8000EA6AF70FE96E020EEA22EF6ADF2AEDD73E
:103F9000010EE66EE66AE66AD10EE66E020EE66E87
:103FA0008DEC35F0146E050EE15E1450609C02013C
:103FB000080EDA6F040EDB6F000ED26F040ED36FA3
:103FC000D2C2D4F2D56F22C4D0F2D05102E1100E89
:103FD00012D0010EE66EE66AD00EE66E020EE66EB6
:103FE000010EE66EE66A30EC1AF0146E060EE15E23
:103FF00014500201200ECF6FE552E552E7CFD9FFF2
:104000001200800E0401205D01E09ED00201C00E6E
:10401000E36F04012351030A57E0010A0CE0030A8D
:1040200001E090D00201180EE06F690EE16F000E02
:10403000E26F120E81D0C10E146E690E156E000E65
:10404000166E22C417F0186A196A030E0C6E0D6AF8
:104050000E6A17C007F018C008F019C009F093ECF9
:1040600033F014500424F36E15500520F46E1650EE
:104070000620F86EF4CFF7FFF3CFF6FF0900F5CF77
:10408000E0F20900F5CFE1F20800F5CFE2F2E0C27C
:10409000F6FFE1C2F7FFE2C2F8FF020EF626000EBD
:1040A000F722F8220800F5CFE4F2E0C2F6FFE1C201
:1040B000F7FFE2C2F8FF030EF626000EF722F82201
:1040C0000800F5CFE5F21200030E225D38E2C40EBF
:1040D000146E690E156E000E166E22C417F0186A63
:1040E000196A030E0C6E0D6A0E6A17C007F018C02D
:1040F00008F019C009F093EC33F014500424F36E67
:1041000015500520F46E16500620F86EF4CFF7FF18
:10411000F3CFF6FF0900F5CFE0F20900F5CFE1F2A9
:104120000800F5CFE2F2E0C2F6FFE1C2F7FFE2C21B
:10413000F8FF0800F5500201E46FE56B1200020180
:10414000E36B12000201E36B1200D9CFE6FFE1CF6F
:10415000D9FF020EE1260401286B296B20511F0BA9
:10416000020A11E0030A0CE0010A3CE10201E38FBC
:10417000040128810201F00535E10401288332D0D1
:104180000201E38F2FD00201E38F040124BF0BD083
:1041900024510F0BE96EEA6AD890E936EA36D60E5A
:1041A000E926020E0AD024510F0BE96EEA6AD89074
:1041B000E936EA36DA0EE926020EEA22EECFDEFF13
:1041C000EDCFDDFFDECFE9FFDDCFEAFFEF50800B63
:1041D00009E0DECFE9FFDDCFEAFFEF50040B02E09C
:1041E000010E286F0201E3AF07D0280EE06F040E26
:1041F000E16FE381020EE46F020EE15C02E2E16A2C
:10420000E552E16EE552E7CFD9FF12006AA015D062
:10421000D2C2E9FFD3C2EAFFEF5080080DE1DAC253
:10422000E9FFDBC2EAFFEF50840806E1D2C2E9FFF2
:10423000D3C2EAFF8C0EEF6E6A90659A1200648416
:10424000659860820201010EF16F000EE66EE66A6B
:10425000E66EE66A750EE66EE66A30EC1AF0146EEB
:10426000060EE15E145012000201F16B000EE66EC4
:10427000E66AE66EE66A740EE66EE66A30EC1AF0FE
:10428000146E060EE15E14506092649465A402D030
:104290006594FCD71200D9CFE6FFE1CFD9FFE652F3
:1042A00002012D0EF96FFD0EF21553E17E0EF2158F
:1042B000E8407F0B040DF3CFD2F2F4CFD3F2000E1F
:1042C000D227040ED323D2C2D4F2D3C2D5F2D475EE
:1042D000D2C2E9FFD3C2EAFFEF503C0BE842E8420A
:1042E0000D0835E1DF6A080EDF5C23E2D2C2E9FF88
:1042F000D3C2EAFF020EE926000EEA22EE50EFCF0B
:10430000EAFFE96EEF50E66EDF50EA6A200FE96ED1
:10431000040EEA22E552E750EF6ED2C2E9FFD3C2A3
:10432000EAFF020EE926000EEA22EE2AEF22DF2A39
:10433000DAD7D2C2E9FFD3C2EAFF020EE926000EA5
:10434000EA22200EEE6E040EED6E0DD807D03AD89C
:1043500005D0FD0EF215040801E159D8E552E552E9
:10436000E7CFD9FF12000201DE6BFA6BFD6BFE6B2B
:10437000F46BDF6BDAC2E9FFDBC2EAFFEF9EDA75AE
:10438000DAC2E9FFDBC2EAFFEF9EDA75D4C2E9FFC9
:10439000D5C2EAFFEF9EE36BE46BE56BE86BE96B7C
:1043A000EA6B8FD8000EE66EE66AE66EE66A030EEA
:1043B000E66EE66A30EC1AF0146E060EE15E1450FA
:1043C0002BEF1EF0020E0201DF5D02E1EEEF1EF0A8
:1043D000DF6BF4511AE1D4C2E9FFD5C2EAFFEE5215
:1043E000080EEF6ED4C2E9FFD5C2EAFF020EE9263D
:1043F000000EEA22200EEE6E040EED6ED4C2E9FF2E
:10440000D5C2EAFF8C0EEF6E1200F46B1200D9CF0A
:10441000E6FFE1CFD9FFE652DAC2E9FFDBC2EAFFED
:10442000EF50400B01E0010EDF6E0201DA75080E5D
:10443000CF5D08E122C463FF635002E0100E01D09B
:10444000040ECF6FDF0526E1DAC2E9FFDBC2EAFF27
:10445000020EE926000EEA22280EEE6E040EED6E24
:104460005BDC020E0201DE5D06E1DAC2E9FFDBC2BF
:10447000EAFF840E0DD0DF5006E1DAC2E9FFDBC2AD
:10448000EAFFC80E05D0DAC2E9FFDBC2EAFF880EF8
:10449000EF6E12D0E8AF0FD0EB51EC11ED1109E047
:1044A00007D0EDC2FBFFECC2FAFF0201EB51F96E3F
:1044B000F8DF0201E89FDF6BE552E552E7CFD9FF55
:1044C000120004012051600BE842E842E842E84251
:1044D000E842000901E0120021510C0A50E00B0AE9
:1044E0003FE00C0A31E0010A22E00B0A1EE0020A5A
:1044F0001CE0030A18E0080A10E0010A0CE00F0AA9
:1045000008E0030A01E012000201E38F080ECF6FFA
:10451000120001EF20F090EF1FF00201D00EE06FCB
:10452000020EE16F0CD0A5EF20F0C0EF22F0245175
:104530000201E06FE16BD10EE027020EE123E3817F
:10454000010EE46FE38F12000201E38F0401245196
:10455000EA6AD10FE96E020EEA2222C4EFFF1200CE
:10456000000EE66EE66AE66EE66A020EE66EE66A41
:1045700030EC1AF0146E060EE15E145012001200B8
:10458000D9CFE6FFE1CFD9FF050EE12604012205D0
:1045900010E120511F0B00090CE10201E38F030E13
:1045A0000401215D04E10201010EF06F02D002015D
:1045B000F06B0401225101E011D120511F0B0208C0
:1045C00001E00CD124510F0B000901E107D1245166
:1045D0000F0B010801E202D1200E0201CF5D01E0C4
:1045E000FDD0E38F040124BF16D024510F0BE96ED8
:1045F000EA6AD890E936EA36D60EE926020EEA22B1
:10460000EECFDEFFEDCFDDFF24510F0BEA6AF70F8F
:10461000E96E020E15D024510F0BE96EEA6AD890AC
:10462000E936EA36DA0EE926020EEA22EECFDEFF9E
:10463000EDCFDDFF24510F0BEA6AF50FE96E020E94
:10464000EA22020EEFCFDBFFD950020FE96EDACF7C
:10465000EAFFEF50010B03E1000EDF9401D0DF848D
:1046600024BF0BD024510F0BE96EEA6AD890E936CB
:10467000EA36D60EE926020E0AD024510F0BE96E57
:10468000EA6AD890E936EA36DA0EE926020EEA221C
:10469000DECFEEFFDDCFEDFF030E215D20E1DECFAB
:1046A000E9FFDDCFEAFFEF50800B11E024BF07D018
:1046B00024510F0BEA6AF70FE96E020E06D024515F
:1046C0000F0BEA6AF50FE96E020EEA22EF82840E02
:1046D000DECFE9FFDDCFEAFFE850EF127FD0DF74D5
:1046E000DECFE9FFDDCFEAFFEF50800B1BE0DECF2E
:1046F000E9FFDDCFEAFFEF9EDECFE9FFDDCFEAFF86
:10470000EF8C020EE66EE66ADECFE6FFDDCFE6FF57
:10471000050EE66EE66A30EC1AF0146E060EE15EE7
:10472000145005D0DECFE9FFDDCFEAFFEF8CDF7458
:10473000D950020FE96EDACFEAFFEF50020B07E122
:10474000DECFE9FFDDCFEAFFEF50800B2BE0040165
:1047500024BF07D024510F0BEA6AF70FE96E020E4F
:1047600006D024510F0BEA6AF50FE96E020EEA2219
:10477000EF923B0E146EDECFE9FFDDCFEAFFE8508B
:10478000EF16020EE66EE66ADECFE6FFDDCFE6FF4D
:10479000050EE66EE66A30EC1AF0146E060EE15E67
:1047A000145007D03B0EDECFE9FFDDCFEAFFE85023
:1047B000EF16040124510F0B156A6A0F146E0F0EC9
:1047C0001522030E14C0DBFF040E15C0DBFF030E21
:1047D000DBCFE9FF040EDBCFEAFFEF90050EE15CD3
:1047E00002E2E16AE552E16EE552E7CFD9FF12003D
:1047F0000120F00000F00000F00000F000000000D8
:1048000000000000000000000000000000000000A8
:10481000000000000000F00000F00000F00000F0D8
:1048200000000F00000F00000F00000F000000004C
:104830000000000000000000000000000000000078
:104840000000000000000F00000F00000F00000F2C
:10485000000000F00000F00000F00000F000000098
:104860000000000000000000000000000000000048
:1048700000000000000000F00000F00000F0000068
:10488000F000000F00000F00000F00000F000000FC
:104890000000000000000000000000000000000018
:1048A000000000000000000F00000F00000F0000DB
:1048B0000F000000F00000F00000F00000F0000029
:1048C00000000000000000000000000000000000E8
:1048D0000000000000000000F00000F00000F00008
:1048E00000F000000F00000F00000F00000F00009C
:1048F00000000000000000000000000000000000B8
:1049000000000000000000000F00000F00000F007A
:10491000000F000000000000000000000000000088
:104920000000000000000000000088888888888857
:1049300088888888888888888888888888888888F7
:10494000888844444444444444444444444444449F
:1049500044444444444444444444222222222222E3
:104960002222222222222222222222222222222227
:104970002222111111111111111111111111111105
:10498000111111111111111111110000000000007D
:104990000000000000000000000000000000000017
:1049A0000000FFFFFF000000000000000000FFFF0C
:1049B000FF000000000000000000000000FFFFFFFB
:1049C000000000000000000000FFFFFF00000000EA
:1049D0000000000000000000FFFFFF0000000000DA
:1049E00000000000FFFFFF000000000000000000CA
:1049F000000000FFFFFF000000000000000000FFBB
:104A0000FFFF0000000000000000000000000000A8
:104A1000000000000000000000000203C00000C011
:104A2000000C00030C000300C00000C0000C0003D9
:104A30000C0003000760000C60000C000300000382
:104A40000060000C60000C003000003000073000F7
:104A50000C30000C0030000030003000C03000C0CE
:104A6000003000003000070300C00300C0006000F9
:104A70000060003000C03000C0006000006000072F
:104A800003006003006000C00000C000030060037A
:104A9000006000C00000C0000700003003C0300309
:104AA000C00000000000003003C03003C000000060
:104AB000000700C00000C03003003003000000C049
:104AC0000000C03003003003000007000C00000CA1
:104AD0000006003006003000C00000C000060030B4
:104AE00006003007000C00000C000C00030C000353
:104AF000000C00000C000C00300C00300700060019
:104B00000006000C00030C0003000600000600C0B5
:104B10000003C0000307000300000300C00006C03C
:104B20000006000300000300C00006C000060700E6
:104B30000000C00300C0030C00000C000000C00314
:104B400000C0030C00000C070101FF0000FF000083
:104B5000FF0000FF0000FF0000FF0000FF0000FF5B
:104B6000000000FF0000FF0000FF0000FF0000FF4A
:104B70000000FF0000FF0000FF000000FF0000FF3A
:104B80000000FF0000FF0000FF0000FF0000FF002A
:104B900000FFFFFF00FFFF00FFFF00FFFF00FFFF20
:104BA00000FFFF00FFFF00FFFF0000FFFF00FFFF0F
:104BB00000FFFF00FFFF00FFFF00FFFF00FFFF00FF
:104BC000FFFFFF00FFFF00FFFF00FFFF00FFFF00F0
:104BD000FFFF00FFFF00FFFF00FFFFFFFFFFFFFFE2
:104BE000FFFFFFFFFFFFFFFFFFFFFFFFFFFFFFFFD5
:104BF000FFFF0000000000000000000000000000B7
:104C0000000000000000000000000204000000009E
:104C10000000000000000000000000000000000094
:104C20000000000007FF0000FF0000FF0000FF0081
:104C300000FF0000FF0000FF0000FF000007000071
:104C40000000000000000000000000000000000064
:104C50000000000000000700FF0000FF0000FF0050
:104C600000FF0000FF0000FF0000FF0000FF000742
:104C70000000000000000000000000000000000034
:104C80000000000000000000070000FF0000FF001F
:104C900000FF0000FF0000FF0000FF0000FF000019
:104CA000FF070000000000000000000000000000FE
:104CB0000000000000000000000007FFFF00FFFFF1
:104CC00000FFFF00FFFF00FFFF00FFFF00FFFF00EE
:104CD000FFFF000700FFFF00FFFF00FFFF00FFFFD7
:104CE00000FFFF00FFFF00FFFF00FFFF07FF00FFC7
:104CF000FF00FFFF00FFFF00FFFF00FFFF00FFFFBF
:104D000000FFFF00FF07FFFFFFFFFFFFFFFFFFFFA9
:104D1000FFFFFFFFFFFFFFFFFFFFFFFFFFFF070298
:104D200040FFFF00FFFF00FFFF00FFFF00FFFF004D
:104D3000FFFF00FFFF00FFFF000300FFFF00FFFF7A
:104D400000FFFF00FFFF00FFFF00FFFF00FFFF006D
:104D5000FFFF03FF00FFFF00FFFF00FFFF00FFFF5B
:104D600000FFFF00FFFF00FFFF00FF0302018010B4
:104D700000000000000000000080000001000000B2
:104D800000000001080007C00001800000000000D2
:104D9000000800800003000001000800000C00076C
:104DA000680003C00001800800000C00C0001680ED
:104DB0000803000C01008600073C0016680803C0C9
:104DC0000C0180860068083CC00C1680860300C376
:104DD000010716083C3C0C16688603C0C301340C5E
:104DE000686C863CC8C31680610307030C6816868E
:104DF0003C3CC3166861031686C03CC36868613CCE
:104E0000C03016070186C003C36816613C3C3016EB
:104E100003C3801661C03C306868103C0700C38043
:104E20000161C003306816103C0161000330801638
:104E300010C03C0068070061000030800110C00312
:104E400000680030000110000300801600C0070059
:104E500030000010000000800100C00010000000C1
:104E600000010000030080070201F00000F00000D4
:104E7000F00000F000000000000000000000000052
:104E8000000007F00000F00000F00000F00000F06B
:104E90000000F00000F00000F0000007FF0000FF3D
:104EA0000000FF0000FF0000F00000F00000F00034
:104EB00000F0000007FF0000FF0000FF0000FF00FF
:104EC00000FF0000FF0000FF0000FF000007EE00F1
:104ED00000EE0000EE0000EE0000EE0000EE00002C
:104EE000EE0000EE000007CC0000CC0000CC00007B
:104EF000CC0000CC0000CC0000CC0000CC000007AF
:104F00008800008800008800008800008800008871
:104F1000000088000088000007000000000000007A
:104F20000000000000000000000000000000000081
:104F300000070088000088000088000088000088C2
:104F4000000088000088000088000700CC0000CC2A
:104F50000000CC0000CC0000CC0000CC0000CC0055
:104F600000CC000700EE0000EE0000EE0000EE00B6
:104F700000EE0000EE0000EE0000EE000700FF0073
:104F800000FF0000FF0000FF0000FF0000FF000026
:104F9000FF0000FF000700000000FF0000FF00000E
:104FA000FF0000000000FF0000FF0000FF000700FE
:104FB000000000000000FF0000FF000000000000F3
:104FC0000000FF0000FF00070000000000000000DC
:104FD0000000FF0000000000000000000000FF00D3
:104FE00007000000000000000000000000000000BA
:104FF00000000000000000000007000000000000AA
:105000000000000000FF00000000000000000000A1
:1050100000FF070000000000000000FF0000FF008C
:1050200000000000000000FF0000FF07000000007B
:1050300000FF0000FF0000FF0000000000FF000074
:10504000FF0000FF070000FF0000FF0000FF00005E
:10505000FF0000FF0000FF0000FF0000FF0700004E
:105060000F00000F00000F00000F0000FF0000FF06
:105070000000FF0000FF0700000F00000F00000FFE
:1050800000000F00000F00000F00000F00000F07CE
:1050900000000000000000000000000000000F0001
:1050A000000F00000F00000F0700000000000000CC
:1050B00000000000000000000000000000000000F0
:1050C00000070000000000000000000000000F00CA
:1050D000000F00000F00000F0000070F00000F007E
:1050E000000F00000F00000F00000F00000F000075
:1050F0000F0000070F00000F00000F00000F00005E
:10510000FF0000FF0000FF0000FF000007FF00009D
:10511000FF0000FF0000FF0000FF0000FF0000FF95
:105120000000FF000007770000770000770000779D
:105130000000770000770000770000770000073359
:105140000000330000330000330000330000330060
:1051500000330000330000071100001100001100AF
:1051600000110000110000110000110000110000EA
:105170000700000000000000000000000000000028
:1051800000000000000000000007001100001100F6
:1051900000110000110000110000110000110000BA
:1051A000110007003300003300003300003300001B
:1051B00033000033000033000033000700770000A5
:1051C0007700007700007700007700007700007715
:1051D000000077000700FF0000FF0000FF0000FF55
:1051E0000000FF0000FF0000FF0000FF000700FFBD
:1051F0000000FF0000FF0000000000FF0000FF00B3
:1052000000FF000000000700FF0000FF000000009A
:1052100000000000FF0000FF000000000000000789
:1052200000FF0000000000000000000000FF000080
:105230000000000000000000070000000000000067
:10524000000000000000000000000000000000005E
:1052500000070000FF000000000000000000000048
:10526000FF000000000000000000070000FF000039
:10527000FF0000000000000000FF0000FF00000031
:10528000000000070000FF0000FF0000FF0000001A
:105290000000FF0000FF0000FF000000070000FF0B
:1052A0000000FF0000FF0000FF0000FF0000FF0003
:1052B00000FF0000FF070000FF0000FF0000FF00EC
:1052C00000FF0000F00000F00000F00000F0070018
:1052D00000F00000F00000F00000F00000F000001E
:1052E000F00000F00000F0070000F00000F0000007
:1052F000F00000F0000000000000000000000000CE
:105300000700000000000000000000000000000096
:10531000000000000000000000070110C00000C0F5
:10532000000C00030C000300C00000C0000C0003D0
:105330000C00030060000C60000C00030000030080
:1053400060000C60000C00300000300030000C30B9
:10535000000C0030000030003000C03000C00030D1
:10536000000030000300C00300C0006000006000C7
:105370003000C03000C00060000060000300600327
:10538000006000C00000C00003006003006000C0B7
:105390000000C00000003003C03003C00000000067
:1053A00000003003C03003C00000000000C0000057
:1053B000C03003003003000000C00000C030030014
:1053C00030030000000C00000C0006003006003026
:1053D00000C00000C000060030060030000C0000D5
:1053E0000C000C00030C0003000C00000C000C006F
:1053F000300C00300006000006000C00030C000317
:10540000000600000600C00003C000030003000007
:105410000300C00006C00006000300000300C00037
:1054200006C00006000000C00300C0030C00000C12
:10543000000000C00300C0030C00000C0202F08852
:10544000FFF08800F08800F088000088FF008800E6
:10545000008800008800070044000044FF0044006A
:10546000004400F04400F044FFF04400F044000722
:105470000F22000F22000F22FF0F22000022000047
:1054800022000022FF00220007001100001100008E
:1054900011000011FF0F11000F11000F11000F116B
:1054A000FF070202F04400F04400F04400F0440022
:1054B000004400004400004400004400070022FFB4
:1054C000002200002200002200F022FFF02200F063
:1054D0002200F02200070F11000F11FF0F11000F23
:1054E00011000011000011FF001100001100070061
:1054F00000000000000000FF0000000F00000F008F
:10550000000F00FF0F00000700FF00000000000078
:10551000000000FF00FF000000000000000000FF8E
:105520000788000088FF00880000880000880000CD
:1055300088FF00880000880000074400F04400F065
:1055400044FFF04400F044000044000044FF0044E5
:1055500000000722000022000022000022FF00229B
:1055600000F02200F02200F022FFF00711000F11DE
:10557000000F11000F11000F1100001100001100A9
:10558000001100000700F00000F00000F00000F043
:105590000000000F00000F00000F00000F07FF00C9
:1055A00000000000000000000000FFF00000F0001C
:1055B00000F00000F00007000F88FF0F88000F8840
:1055C000000F88000088FF0088000088000088071E
:1055D000000044000044FF0044000044000F440069
:1055E0000F44FF0F44000F44070000220000220078
:1055F0000022FF0022000022000022000022FF0003
:105600002207008811008811008811008811008885
:105610001100881100881100881107030107031089
:105620000703200204040F02010000000000000034
:10563000000000000000000000000000000000006A
:10564000001F00000006000006000000000000002F
:1056500000000000600000600000070600006F000E
:10566000006F0000060000600000F60000F6000079
:10567000600000026F0000FF0000FF00006F0000EC
:10568000F60000FF0000FF0000F6000002FF00002F
:10569000FF0000FF0000FF0000FF0000FF0000FF10
:1056A0000000FF000003FF0000F90000F90000FF08
:1056B0000000FF00009F00009F0000FF000002F9B3
:1056C0000000900000900000F900009F0000090019
:1056D000000900009F000002000000000000000020
:1056E00000000000000000000000000000000000BA
:1056F0003F0000000006000006000000000000005F
:1057000000600000600000000007000600006F005D
:10571000006F0000060000600000F60000F60000C8
:10572000600002006F0000FF0000FF00006F00003B
:10573000F60000FF0000FF0000F6000200FF00007E
:10574000FF0000FF0000FF0000FF0000FF0000FF5F
:105750000000FF000300FF0000F90000F90000FF57
:105760000000FF00009F00009F0000FF000200F902
:105770000000900000900000F900009F0000090068
:10578000000900009F00020000000000000000006F
:105790000000000000000000000000000000003FCA
:1057A00000000000000600000600000000000000ED
:1057B00000600000600000000700000600006F00AD
:1057C000006F0000060000600000F60000F6000018
:1057D000600200006F0000FF0000FF00006F00008B
:1057E000F60000FF0000FF0000F6020000FF0000CE
:1057F000FF0000FF0000FF0000FF0000FF0000FFAF
:105800000000FF030000FF0000F90000F90000FFA6
:105810000000FF00009F00009F0000FF020000F951
:105820000000900000900000F900009F00000900B7
:10583000000900009F0200000000000000000000BE
:1058400000000000000000000000000000001F2A0F
:10585000022E01C20015014D00FC00B204220166B7
:10586000007901030003000300030028020614FF6F
:0C5870000A0A1E0614320CFF40404005DE
:04587C007AEC31F0A1
:10588000FB0EDBCFF3FFDB06F35000090AE0C8ECA8
:1058900031F0FA0E33EC32F0F3E1151CF1E1010EB8
:1058A00001D0000EA9EF31F07AEC31F03B0EE1248B
:1058B00002E3E168E652E16E010EDB6A020EDB6A8A
:1058C000F90EDBCFF6FFFA0EDBCFF7FFFB0EDBCFD7
:1058D000F8FF0800F550DF6EDF5002E1CDEF30F049
:1058E000250EDF5C02E0C0EF30F0030EDB6A040E31
:1058F000DB6A050EDB6A060EDB6A070EDB6AE2EC8A
:1059000030F02D0EDF5C0CE02B0EDF5C09E0200E8A
:10591000DF5C06E0230EDF5C03E0300EDF5C1AE1A3
:10592000DF50300A14E0130A0FE0030A0AE00B0A02
:1059300005E0060AE4E1030EDB80E1D7030EDB821B
:10594000DED7030EDB84DBD7030EDB86D8D7030E4E
:10595000DB88D5D72A0EDF5C1BE1DEEC30F02CECC7
:1059600031F010E0030EDB8008680968130EDBCF0E
:105970000DF0140EDBCF0EF0FAEC33F0040E06C07F
:10598000DBFF03D0130E15EC31F0E2EC30F00BD05E
:10599000090EDB6A83EC31F003E0F7EC31F0FAD763
:1059A000090E15EC31F0030EDBB0DB982E0EDF5C38
:1059B0001BE1E2EC30F02A0EDF5C0BE1DEEC30F0B4
:1059C0002CEC31F003E1130E67EC31F0E2EC30F037
:1059D0000BD0090EDB6A83EC31F003E0F7EC31F019
:1059E000FAD7090E67EC31F0680EDF5C07E1E2ECF4
:1059F00030F0680EDF5C1DE1030E18D0740EDF5C22
:105A000017E07A0EDF5C14E0480EDF5C06E0540E0F
:105A1000DF5C03E05A0EDF5C02E1020E07D06C0E81
:105A2000DF5C03E06A0EDF5C04E1010EBAEC31F0EA
:105A3000C9DBDF506E0A01E17FD31E0A01E192D17A
:105A4000200A01E18FD13F0A01E149D11A0A01E19F
:105A500046D10D0A01E143D1200A01E140D13A0AC1
:105A600001E13DD1200A01E13AD1260A01E135D117
:105A70000D0A01E132D11A0A01E1D9D0200A4AE027
:105A8000300A1FE0460A0EE0250A01E083D3D95010
:105A9000F90FE96EFF0EDA20EA6E010EEE5E000EDF
:105AA000EE5AEE5AC8EC31F0250EE66E95DB03E1B6
:105AB000151C01E169D3C4EC31F001E26BD3DB2AA0
:105AC00069D3080EDB6A040EDB50010806E2040EFF
:105AD000DB048CEC31F0DB508BDB080EDB5009E093
:105AE000030EDB50010B05E172DB01E04DD3080E24
:105AF000DB6A64DBEFCFDFFF3CEC32F003E1151C27
:105B000001E142D3C4EC31F001E3DB2A60DB01E1C7
:105B100041D33AD3070EDB5002080FE108EC32F014
:105B2000030ECFEC31F00E0EEECFDBFF0F0EEECFFB
:105B3000DBFF100EEECFDBFF20D0F70EDBCF17F030
:105B4000F80EDBCF18F0020E175E000E185AF70E93
:105B500017C0DBFFF80E18C0DBFF17C0E9FF18C045
:105B6000EAFFBFEC31F0166A0E0E14C0DBFF0F0E19
:105B700015C0DBFF100E16C0DBFF0E0EDBCFE6FFFD
:105B80000F0EDBCFE6FF100EDBCFE6FFB5EC35F0F6
:105B9000E552E552E552130E07C0DBFF140E08C0B4
:105BA000DBFF060EDB5005E0130E03EC32F001E2E2
:105BB0006ADB27EC32F002E2130E37DBEAEC31F05D
:105BC00006E0040E03EC32F002E2050E2EDB030EBB
:105BD000DBB005D0FCDA01E0D7D2080EDB6A090E93
:105BE000DB6A0E0EDBCFF6FF0F0EDBCFF7FF100EDA
:105BF000DBCFF8FF0800F550DF6EDF5014E02DEC2E
:105C000032F011E23CEC32F003E1151C01E1BCD2B0
:105C1000BBDB01E3DB2A090EDB2AD9500E0FE96E4C
:105C2000000ECBDBE7D7D3DA01E1B4D2ADD2C6DACE
:105C3000110EEECFDBFF120EEDCFDBFF110EDBCF2F
:105C4000E6FF120EDBCFE6FFA7EC35F0E552E5529A
:105C5000130EF3CFDBFF140EF4CFDBFF060EDB5089
:105C600004E0130ED0DB01E20EDB27EC32F002E29F
:105C7000130EDBDAAFDB05E0040EC5DB02E2050E36
:105C8000D4DA030EDBB005D0A2DA01E07DD2080E33
:105C9000DB6A090EDB6A110EDBCFE9FF120EDBCFE8
:105CA000EAFFEFCFDFFFDF5014E0D7DB12E2E4DBE7
:105CB00003E1151C01E168D267DB01E3DB2A090E71
:105CC000DB2A110EDB2ADBCFE9FF120EE8E3DB2A29
:105CD000E6D77DDA01E15ED257D2030EDB8E070EE6
:105CE000DB0410E195DB040E5ADB0A0EEECFDBFF7E
:105CF0000B0EEECFDBFF0C0EEECFDBFF0D0EEECF6B
:105D0000DBFF6CD0070EDB5003082CE1030EDBAE8B
:105D10000DD0B2DA020E76DAEFCF14F0156A166AF9
:105D2000176A14AE39D01568166835D0F70EDBCF78
:105D300015F0F80EDBCF16F0020E155E000E165AA7
:105D4000F70E15C0DBFFF80E16C0DBFF15C0E9FF2C
:105D500016C0EAFFEFCF14F00A0E14C0DBFF0B0EE3
:105D6000DB6A38D0070EDB50020809E1030EDBAE18
:105D700004D059DB16AE10D00ED055DB0DD0030E7B
:105D8000DBAE12D079DA020E3DDAF9DA166A176A5A
:105D900015AE02D016681768E2DA0C0E16C0DBFFEB
:105DA0000D0E17C0DBFF1AD0F70EDBCF16F0F80E82
:105DB000DBCF17F0020E165E000E175AF70E16C054
:105DC000DBFFF80E17C0DBFF16C0E9FF17C0EAFFC4
:105DD000D6DAC5DA0C0EDB6A0D0EDB6A060EDB5076
:105DE00005E1010EF36E050EF3CFDBFF150EDB6A46
:105DF000160EDB6AD950370F146E000EDA20156EBE
:105E0000390E14C0DBFF3A0E15C0DBFF380EDB6A1B
:105E1000080EDB6A0A0EAEDADF50780A12E0200ABA
:105E200010E0280A0CE0200A0AE03F0A06E00D0A0A
:105E300002E0200A08E1020E05D0080E03D0080E89
:105E4000DF26100E97DA030EDBBE02D0DB92DB9466
:105E5000DB50800B24E08ADAD890030EEB50000A66
:105E600008E6000EEE5C000EEE58000EEE58000E36
:105E7000EE5815E213DA0B680C680D680E685DECDD
:105E800036F00A0E02C0DBFF0B0E03C0DBFF0C0E68
:105E900004C0DBFF0D0E05C0DBFF2D0E08D0030E86
:105EA000DBA202D02B0E03D0DBA408D0200EF36EB1
:105EB000170EF3CFDBFF150EDB2A02D0170EDB6ABD
:105EC000050EDB5003E1B7D901E189D0A00E146EB5
:105ED0006F0E156E000E166E070EDBCF17F0186AE8
:105EE000196A1A6A17C00BF018C00CF019C00DF02F
:105EF0001AC00EF0D3D9FAEC36F014500224F36E27
:105F000015500320F46E16500420F86EF4CFF7FFFE
:105F1000F3CFF6FF0800090EF5CFDBFF580EDF5C6C
:105F20000FE1610EF36E090E7BD90AE3200E146EA9
:105F3000090EDBCFE7FF1450E75E090EE7CFDBFF6A
:105F4000070EDBCF14F0156A166A176A0FDA14C051
:105F50000BF015C00CF016C00DF017C00EF0EECF10
:105F600006F0EECF07F0EECF08F0EFCF09F0FAEC35
:105F700036F009C0EDFF08C0EDFF07C0EDFF06C019
:105F8000EFFF390EDBCFE9FFDB063A0EDBCFEAFF8E
:105F900001E2DB06090EDBCFEFFF150EDB2A4BD942
:105FA00095E1030EDBA61DD06F0EDF5C06E1C1D9C3
:105FB00018E3150EDB285BDA14D0780EDF5C09E0FD
:105FC000580EDF5C06E0620EDF5C03E0420EDF5C31
:105FD00008E1020EF36E160EF3CFDBFF02D0150EB2
:105FE000DB6A030EDB50100B0EE0040EDBCF14F067
:105FF000050EDB50D880145406E2060EDB5003E198
:10600000040EDB5034DA95D90AE2050EDBCFE7FF48
:10601000150EDB50E75E050EE7CFDBFF02D0050E65
:10602000DB6A040EDBCF14F0160E45D9D880145469
:1060300014E2160EDBCFE6FF150EDBCFE6FF040EF3
:10604000DBCFE6FF050EDB50E552E75CE552D8807A
:10605000E754E552D880E7545FD9030EDB50010BBB
:106060000BE1080EDB5008E0B2D801E08DD0080E3D
:10607000DB50BED8080EDB6A170EDB5007E088D96C
:10608000170EF1D903E1151C01E17ED0160EDB508D
:1060900016E07ED9300EE66E9FD802E1151C74E042
:1060A00077D9DFCFE6FFDAEC35F0E552E552E5527D
:1060B000F4CF15F00001F31C02E1151C65E0050E9C
:1060C000DBCF14F0160EDB50D880145409E2050E15
:1060D000DBCFE7FF160EDB50E75E050EE7CFDBFFF9
:1060E000300EE66E050ECBD94FE1390EDB2ADBCF41
:1060F000E9FF3A0E01E3DB2ADBCFEAFF090EEFCF1F
:10610000DBFFDB500EE044D9090EADD902E1151CCE
:106110003BE0390EDB2ADBCFE9FF3A0EEDE3DB2A69
:10612000EBD755D831E1160EDBCFE6FF080EC3D80A
:10613000E552E7245DD82ED0070EDB50030A1CE0A1
:10614000010A14E0030A07E07BD9DBCFEEFF020E61
:10615000DBCFEDFF1FD0F5D8196A17AE02D0186853
:1061600019682CD8BCD819C0EEFF14D0EAD817BED5
:10617000186824D8B4D80ED063D9DBCFEFFF0AD08B
:106180007BD905E1151C03E1F368F46810D0FCD855
:1061900001E3DB2A79D969EF2CF0010EDBCF14F093
:1061A000020EDBCF15F014C0F3FF15C0F4FF3B0E59
:1061B000E15C02E2E16AE552E16ECBD029D9020E40
:1061C000CFEF31F061D90800F550DF6E1200200EDC
:1061D000E66E080E3FEF32F0DAEC35F0E552E552AC
:1061E000E552F3CF14F0F4CF15F00001F31C1200C8
:1061F000146E156AD950010F4DD91450EE26155062
:10620000ED221200185E000E195AF70E18C0DBFFBF
:10621000F80E19C0DBFF18C0E9FF19C0EAFF120031
:10622000DBCFF4FFF350F45C1200DB50E76E040E9A
:10623000E7CFDBFF12000A0EDBCF14F00B0EDBCF33
:1062400015F00C0EDBCF16F00D0EDBCF17F014504F
:106250001510161017101200130EEECFDBFF140EE0
:10626000EDCFDBFF130EDBCF14F0140EDBCF15F0F8
:106270000001800E15141200F70EDBCF18F0F80E97
:10628000DBCF19F01200050EDB50E66ED950130F6C
:1062900001D9E552E750EE6EED6A12000A0EDBCF2F
:1062A00006F00B0EDBCF07F00C0EDBCF08F00D0E67
:1062B000DBCF09F01200DBCFE6FF150EDBCFE6FFE8
:1062C000050EDB50E552E724E552E7241200DB50CF
:1062D000CED8010EF36E060EF3CFDBFF1200EE50A8
:1062E000EFCFEAFFE96E16C0EEFF17C0EEFF18C051
:1062F000EEFF1200D9CFE6FFDACFE6FFE1CFD9FFFC
:10630000E2CFDAFF1200DFCFE6FFE66A92EC37F069
:10631000E552E552F3501200E76E080EE7CFDBFFBF
:106320001200EECF14F0EECF15F0EFCF16F0176A93
:106330001200050EDBCF14F0150EDB50D88014547C
:106340001200010EDBCF16F0020EDBCF17F0186A39
:106350001200E552E5CFDAFFE7CFD9FF12000A0EAF
:1063600014C0DBFF0B0E15C0DBFF1200D9500A0F63
:106370004AEF32F0F36E070EF3CFDBFF1200EECFE1
:1063800014F0EFCF15F01200010EDB2A020E1200FE
:10639000FC0EDBCFE6FFFD0EDBCFE6FF1200145E46
:1063A000000E155AF70E14C0DBFFF80E15C0DBFF08
:1063B00014C0E9FF15C0EAFF1200DA20EA6EEF2AE6
:1063C000EECFF6FF000EEF22EECFF7FFEF22EECF7B
:1063D000F8FF1200040EDBCFE6FF130EDB50E55290
:1063E000E75C9ADFDB5004DF060EDB501200090E7B
:1063F000DB500A0DF350DF24D00FE76E090EE7CF14
:10640000DBFFE2EF30F0DB50F36E050E10EF31F002
:10641000F70EDBCF14F0F80EDBCF15F01200DFCF54
:10642000E6FFECEF30F028DF030EECDE91EF31F009
:106430003EEC2CF0E552E552E552E552000912001F
:10644000BDDEEE50EFCFEAFFE96E010E1200130E33
:10645000DB50F36E040E10EF31F0040EDB50F36EE0
:10646000090E10EF31F0DBCFE6FFECEF30F0E76E16
:10647000050EE7CFDBFF12008BDF0FEF32F0DBCF33
:10648000E6FF86DF18EF32F0D950F90FE96EFF0E04
:0E649000DDEF31F0E96E000EDA20EA6E120048
:02649E000001FB
:1064A000606B616B626B636B646B656B1200D9CF61
:1064B000E6FFE1CFD9FF020EE126FD0EDBCFE6FFBE
:1064C000FE0EDBCFE6FFA7EC35F0E552E55200010A
:1064D0006451F324146E6551F420156E820E145C21
:1064E000000E155801E396D0DE6ADD6ADECF14F0A7
:1064F000DDCF15F014C0E6FF15C0E6FFFD0EDBCFC3
:10650000E6FFFE0EDBCFE6FFA7EC35F0E552E552E5
:10651000E552E7CF15F0E552E7CF14F0F3CF16F0D0
:10652000F4CF17F0F350145CF450155834E2FD0E1C
:10653000DBCF14F0FE0EDBCF15F0DE501424E96E35
:10654000DD501520EA6EEF50E66E660E0001622502
:10655000E96E000E6321EA6EE552E750EF6E010E20
:106560006225626F000E6321636F840E0D6E0E6AEA
:1065700062C008F063C009F07CEC37F004C062F040
:1065800005C063F00001642B000E6523DF2A010EB5
:10659000ADE3DB2AABD7660E00016225E96E000E83
:1065A0006321EA6E0D0EEF6E010E6225626F000E22
:1065B0006321636F840E0D6E0E6A62C008F063C0C3
:1065C00009F07CEC37F004C062F005C063F0000114
:1065D000642B000E6523660E0424E96E000E052070
:1065E000EA6E0A0EEF6E010E6225626F000E6321E5
:1065F000636F840E0D6E0E6A62C008F063C009F00E
:106600007CEC37F004C062F005C063F00001642B3D
:10661000000E6523020EE15C02E2E16AE552E16EE2
:10662000E552E7CFD9FF1200D9CFE6FFE1CFD9FF7E
:10663000040EE126DE6ADD6A00013F0ED880645553
:10664000000E655504E23F0EDE6EDD6A04D064C0C4
:10665000DEFF65C0DDFFDECF14F0DDCF15F01406E0
:10666000000E155AFD0EDBCFE9FFFE0EDBCFEAFF71
:1066700014C0EFFF645165114CE0010EF36E020E81
:10668000F3CFDBFF030EDB6A020EDBCF14F0030E49
:10669000DBCF15F0DECF16F0DDCF17F01650145C0F
:1066A0001750155836E2660E6025E96E000E61211E
:1066B000EA6EEF50E66E020EDBCF14F0030EDBCF76
:1066C00015F0FD0EDB501424E96EFE0EDB50152094
:1066D000EA6EE552E750EF6E010E6025606F000E26
:1066E0006121616F840E0D6E0E6A60C008F061C09A
:1066F00009F07CEC37F004C060F005C061F00001E7
:106700006407000E655B020EDB2A030EBDE3DB2A85
:10671000BBD7040EE15C02E2E16AE552E16EE552AC
:06672000E7CFD9FF1200D3
:0A67260009C013F008C012F007C00C
:1067300011F007500C02F4CF05F0F3CF04F008502D
:106740000D02F4CF07F0F3CF06F00C02F35005264C
:10675000F4500622E86A072211500D02F350052674
:10676000F4500622E86A072209500C02F35006266C
:10677000F450072209500D02086AE86A0822F35013
:106780000726F450082211500E02F3500626F4504A
:106790000722096AE86A0822092212500E02F35001
:1067A0000726F4500822E86A092213500E02F3501B
:1067B0000826F4500922000C08C012F008500D02FF
:1067C000F4CF07F0F3CF06F009500E02F4CF09F032
:1067D000F3CF08F00D02F3500726F4500822E86AC0
:1067E000092212500E02F3500726F4500822E86ADC
:1067F0000922000C09C013F008C012F008500D0265
:10680000F4CF07F0F3CF06F009500E02F4CF09F0F1
:10681000F3CF08F00D02F3500726F4500822E86A7F
:10682000092212500E02F3500726F4500822E86A9B
:1068300009220EAE20EF34F01250085E1350095AB0
:0E68400013AE000C0D50085E0E50095A000CED
:02684E00040143
:1068500020511F0B010801E01200245101E0120039
:10686000060E215D1FE12351230A1CE0010A0EE000
:10687000030A18E10201D00515E102013C0EE06FA8
:10688000690EE16F000EE26F090E08D00201A50E3D
:10689000E06F690EE16F000EE26F1C0EE46FE56BB6
:1068A000C00EE36F04012051600BE842E842E84269
:1068B000E842E842010801E0120021510B0A26E0FB
:1068C000080A19E0090A11E0080A05E00B0A23E0AA
:1068D000080A21E012000201F60EE06F000EE16FDF
:1068E000010EE46FE56BC10E0FD00201800EE36F65
:1068F00023C4F6F012000201F70EE06F000EE16F04
:10690000010EE46FE56B810EE36F12000201800E51
:08691000E36F22C4F7F012004E
:0869180012010002000000085A
:10692000D80442000200010203010902290001010A
:1069300000C0320904000002030000000921110117
:106940000001221C00070581034000010705010327
:10695000400001040309041603320044004B00699F
:1069600000740073002E0063006F006D002C033272
:106970000044004B006900740073002E0063006F38
:10698000006D0020003400780034007800340020CE
:106990000063007500620065000C03560030002E95
:1069A00000300031000600FF0901A1011901294052
:1069B0001501254075089540810019012940910075
:1069C000C02A69005369005769006D690099690020
:1069D000D9CFE6FFDACFE6FFE1CFD9FFE2CFDAFF8A
:1069E000E652E652E652E652D950F90F146EFF0E07
:1069F000DA20156E020E14C0DBFF030E15C0DBFF9C
:106A0000020EDBCFE6FF030EDBCFE6FFF90EDBCF96
:106A1000E6FFFA0EDBCFE6FFFB0EDBCFE6FFD95039
:106A2000FC0FE66EFF0EDA20E66E54EC2CF0146ECE
:106A3000070EE15C02E2E16AE552E16E1450F3CF29
:106A4000DEFFF4CFDDFFFC0EDBCFE9FFFD0EDBCF79
:106A5000EAFFEF6ADECF14F0DDCF15F014C0F3FFCC
:106A600015C0F4FF040EE15C02E2E16AE552E16E5A
:0C6A7000E552E5CFDAFFE7CFD9FF1200B6
:046A7C001E0EF66E86
:106A8000000EF76E000EF86E00010900F550EF6F72
:106A90000900F550F06F03E1EF6701D03DD0090028
:106AA000F550EA6F0900F550EB6F0900F550EC6FF7
:106AB00009000900F550E96E0900F550EA6E090079
:106AC00009000900F550ED6F0900F550EE6F09005F
:106AD0000900F6CFF1F0F7CFF2F0F8CFF3F0EAC00B
:106AE000F6FFEBC0F7FFECC0F8FF0001ED5302E149
:106AF000EE5307E00900F550EE6EED07F8E2EE0701
:106B0000F9D7F1C0F6FFF2C0F7FFF3C0F8FF0001BC
:0A6B1000EF07000EF05BBFD7120084
:066B1A00FE0EE3CFE9FFCF
:106B2000FF0EE3CFEAFFE9CFF3FFEACFF4FFFB0E5E
:106B3000E35003E1FC0EE35009E0FB0EE30602E242
:106B4000FC0EE306FD0EE350EE6EF1D71200FE0ED2
:106B5000E3CFE9FFFF0EE3CFEAFFF36AF46AEE52F8
:106B600003E0F34AF42AFBD71200FF0EE3CFF8FF4D
:106B7000E552FF0EE3CFF7FFE552FF0EE3CFF6FF3E
:106B8000E552E66AE66AE66A0900F55209E0FD0E9A
:106B9000E32A05E1FE0EE32A02E1FF0EE32AF4D721
:106BA000FD0EE3CF07F0FE0EE3CF08F0FF0EE3CFBC
:046BB00009F01200D6
:0C6BB400D9CFE6FFDACFE6FFE1CFD9FF32
:106BC000E2CFDAFFFB0EDBCF14F0FC0EDBCF15F0CB
:106BD0000001800E15141AE1FB0EDBCFE9FFFC0E5D
:106BE000DBCFEAFFEECFF3FFEDCFF4FFEE2A000E8E
:106BF000EF22F3CFE9FFF4CFEAFFFD0EDBCFEFFF8B
:106C0000EF50156AF36E15C0F4FF10D0FB0EDB5089
:106C1000FE0806E1FD0EDBCFE6FFC2EC37F005D043
:106C2000FD0EDBCFE6FF03EC00F0E552E552E5CFC9
:086C3000DAFFE7CFD9FF1200E3
:086C3800546F67676C65204C86
:106C4000454420256400446F776E20746F20706186
:106C5000747465726E20256420256400557020745C
:106C60006F207061747465726E2025642025640045
:106C70007061747465726E2025642025640055531C
:106C8000422044657669636520496E697469616C68
:106C9000697365642E0032444B6974733A2034780A
:106CA0003478342052474220637562652032344B79
:096CB00035302076313430390012
:066CBA0006500B02F3CFAF
:106CC00002F0F4CF03F00C02F3500326000EF42080
:106CD000046E06500D02F3500426000EF420056EDB
:106CE00006500E02F350052607500B02F350032600
:106CF000F4500422000E052207500C02F350042623
:106D0000F450052207500D02F350052608500B02DF
:106D1000F3500426F450052208500C02F3500526C7
:0A6D200009500B02F3500526120083
:066D2A00D9CFE6FFDACF2D
:106D3000E6FFE1CFD9FFE2CFDAFFE652DF6AFF0ECE
:106D4000E76EFC0EDBCF14F0E75014161450A96E5A
:106D5000FB0EDB50A86EA69EA69CA684F250800B6C
:106D600001E0010EDF6EF29E550EA76EAA0EA76E11
:106D7000A682A6B2FED7DF50E8B0F28EE8A0F29E5F
:106D8000A694E552E552E5CFDAFFE7CFD9FF12002E
:106D9000D9CFE6FFDACFE6FFE1CFD9FFE2CFDAFFC6
:106DA0003F0EC716C66AFD0EDB50C612FB0EDB5047
:106DB000C712FC0EDB50030A09E0010A04E0020AD4
:106DC00006E1C78C04D0C78CC68801D0C688FD0EEA
:106DD000DB50050A03E0010A03E1928A938401D0A3
:106DE000939493809396C68AE552E5CFDAFFE7CF76
:046DF000D9FF1200B5
:0C6DF400056A046A036A026A200EE76E5A
:106E0000D890063607360836093602360336043679
:106E100005360B50025C0C5003580D5004580E50B0
:106E2000055809E30B50025E0C50035A0D50045AEA
:0C6E30000E50055A062AE72EE4D7120087
:046E3C00D9CFE6FFC5
:106E4000DACFE6FFE1CFD9FFE2CFDAFFFF0EE76E40
:106E5000FC0EDBCF14F0FD0EDBCF15F0E75014165F
:106E6000156A1450A96EA69CA69EA680000000007C
:106E7000A85000D0E552E5CFDAFFE7CFD9FF1200E6
:106E8000FE0EE3CFF4F0FF0EE3CFF5F01200F5C0F5
:106E900009F0F4C008F0350E0D6E450E0E6EDCECF8
:106EA00033F0062AE86A0722079E07C0F5F006C0FD
:0C6EB000F4F0F4C0F3FFF5C0F4FF120092
:046EBC00D9CFE6FF45
:106EC000DACFE6FFE1CFD9FFE2CFDAFFE652C950D1
:106ED000DF6E9E96C69EFD0EDB50C96EC6AE02D01A
:106EE000FF0E03D09EA6FED7000EE552E552E5CF79
:086EF000DAFFE7CFD9FF120021
:086EF800056A046A100EE76E42
:106F0000D89008360936043605360D50045C0E500C
:106F1000055805E30D50045E0E50055A082AE72E69
:046F2000F0D7120094
:0C6F2400F36AF46AFF0EE124E96EFF0E30
:106F3000E220EA6EED6607D02F0EEF6404D03A0E21
:086F4000EF6001D0F32A1200FA
:086F4800000EF36E00EE00F0F4
:106F5000080E01D81200EA6002D0EE6AFCD7F350A6
:086F6000E9601200EE6AFCD7A3
:086F680013EE00F023EE00F02F
:106F7000F86A019C3EEC35F00AEC00F0EDEC00F014
:046F8000FBD7120029
:0C6F8400FF0EE350ACBA04D0AF6AAB8E35
:106F9000AC8A949CACA2FED7AD6EF36EF46A12007C
:106FA000303132333435363738396162636465667F
:016FB00000E0
:0F6FB100F047001A4A00484B000A4C001F4D00E1
:106FC0006C4D00684E001A53003C5400A254001B44
:0E6FD00056001E56002156002456002756007B
:026FDE000000B1
:106FE000000100000000000000010000010100009D
:0B6FF0000000000000000000E1AC0009
:020000040030CA
:0100000023DC
:0100010028D6
:010002005F9E
:010003003CC0
:0100050001F9
:010006008178
:010008000FE8
:01000900C036
:01000A000FE6
:01000B00E014
:01000C000FE4
:01000D0040B2
:00000001FF
